:020000040000fa
:080000000002040000000000f2
:020000040000fa
:04000800e20300000f
:020000040000fa
:04000c00fc030000f1
:020000040000fa
:04001000ae0300003b
:020000040000fa
:0400140016040000ce
:020000040000fa
:0400180030040000b0
:020000040000fa
:04001c007a03000063
:020000040000fa
:04002000c803000011
:020000040000fa
:040024009403000041
:020000040000fa
:04002800dc040000f4
:020000040000fa
:04002c006e0400005e
:020000040000fa
:04003000dc040000ec
:020000040000fa
:04003400dc040000e8
:020000040000fa
:04003800dc040000e4
:020000040000fa
:04003c00dc040000e0
:020000040000fa
:04004000dc040000dc
:020000040000fa
:04004400dc040000d8
:020000040000fa
:04004800dc040000d4
:020000040000fa
:04004c00dc040000d0
:020000040000fa
:04005000dc040000cc
:020000040000fa
:04005400dc040000c8
:020000040000fa
:04005800dc040000c4
:020000040000fa
:04005c00dc040000c0
:020000040000fa
:04006000dc040000bc
:020000040000fa
:04006400dc040000b8
:020000040000fa
:04006800dc040000b4
:020000040000fa
:04006c00dc040000b0
:020000040000fa
:04007000dc040000ac
:020000040000fa
:04007400dc040000a8
:020000040000fa
:04007800dc040000a4
:020000040000fa
:04007c00dc040000a0
:020000040000fa
:04008000dc0400009c
:020000040000fa
:04008400dc04000098
:020000040000fa
:04008800dc04000094
:020000040000fa
:04008c00dc04000090
:020000040000fa
:04009000dc0400008c
:020000040000fa
:04009400dc04000088
:020000040000fa
:04009800dc04000084
:020000040000fa
:04009c00dc04000080
:020000040000fa
:0400a000dc0400007c
:020000040000fa
:0400a400dc04000078
:020000040000fa
:0400a800dc04000074
:020000040000fa
:0400ac00dc04000070
:020000040000fa
:0400b000dc0400006c
:020000040000fa
:0400b400dc04000068
:020000040000fa
:0400b800dc04000064
:020000040000fa
:0400bc00dc04000060
:020000040000fa
:0400c000dc0400005c
:020000040000fa
:0400c400dc04000058
:020000040000fa
:0400c800dc04000054
:020000040000fa
:0400cc00dc04000050
:020000040000fa
:0400d000dc0400004c
:020000040000fa
:0400d400dc04000048
:020000040000fa
:0400d800dc04000044
:020000040000fa
:0400dc00dc04000040
:020000040000fa
:0400e000dc0400003c
:020000040000fa
:0400e400dc04000038
:020000040000fa
:0400e800dc04000034
:020000040000fa
:0400ec00dc04000030
:020000040000fa
:0400f000dc0400002c
:020000040000fa
:0400f400dc04000028
:020000040000fa
:0400f800dc04000024
:020000040000fa
:0400fc00dc04000020
:020000040000fa
:04010000dc0400001b
:020000040000fa
:04010400dc04000017
:020000040000fa
:04010800dc04000013
:020000040000fa
:04010c00dc0400000f
:020000040000fa
:04011000dc0400000b
:020000040000fa
:04011400dc04000007
:020000040000fa
:04011800dc04000003
:020000040000fa
:04011c00dc040000ff
:020000040000fa
:04012000dc040000fb
:020000040000fa
:04012400dc040000f7
:020000040000fa
:04012800dc040000f3
:020000040000fa
:04012c00dc040000ef
:020000040000fa
:04013000dc040000eb
:020000040000fa
:04013400dc040000e7
:020000040000fa
:04013800dc040000e3
:020000040000fa
:04013c00dc040000df
:020000040000fa
:04014000dc040000db
:020000040000fa
:04014400dc040000d7
:020000040000fa
:04014800dc040000d3
:020000040000fa
:04014c00dc040000cf
:020000040000fa
:04015000dc040000cb
:020000040000fa
:04015400dc040000c7
:020000040000fa
:04015800dc040000c3
:020000040000fa
:04015c00dc040000bf
:020000040000fa
:04016000dc040000bb
:020000040000fa
:04016400dc040000b7
:020000040000fa
:04016800dc040000b3
:020000040000fa
:04016c00dc040000af
:020000040000fa
:04017000dc040000ab
:020000040000fa
:04017400dc040000a7
:020000040000fa
:04017800dc040000a3
:020000040000fa
:04017c00dc0400009f
:020000040000fa
:04018000dc0400009b
:020000040000fa
:04018400dc04000097
:020000040000fa
:04018800dc04000093
:020000040000fa
:04018c00dc0400008f
:020000040000fa
:04019000dc0400008b
:020000040000fa
:04019400dc04000087
:020000040000fa
:040198004a04000015
:020000040000fa
:04019c00dc0400007f
:020000040000fa
:0401a000dc0400007b
:020000040000fa
:0401a400dc04000077
:020000040000fa
:0401a800dc04000073
:020000040000fa
:0401ac00dc0400006f
:020000040000fa
:0401b000dc0400006b
:020000040000fa
:0401b400dc04000067
:020000040000fa
:0401b800dc04000063
:020000040000fa
:0401bc00dc0400005f
:020000040000fa
:0401c000dc0400005b
:020000040000fa
:0401c400dc04000057
:020000040000fa
:0401c800dc04000053
:020000040000fa
:0401cc00dc0400004f
:020000040000fa
:0401d000dc0400004b
:020000040000fa
:0401d400dc04000047
:020000040000fa
:0401d800dc04000043
:020000040000fa
:0401dc00dc0400003f
:020000040000fa
:0401e000dc0400003b
:020000040000fa
:0401e400dc04000037
:020000040000fa
:0401e800dc04000033
:020000040000fa
:0401ec00dc0400002f
:020000040000fa
:0401f000dc0400002b
:020000040000fa
:0401f400dc04000027
:020000040000fa
:0401f800dc04000023
:020000040000fa
:0401fc00dc0400001f
:020000040000fa
:04020000dc0400001a
:020000040000fa
:04020400dc04000016
:020000040000fa
:04020800dc04000012
:020000040000fa
:04020c00dc0400000e
:020000040000fa
:04021000dc0400000a
:020000040000fa
:04021400dc04000006
:020000040000fa
:04021800dc04000002
:020000040000fa
:04021c00dc040000fe
:020000040000fa
:04022000dc040000fa
:020000040000fa
:04022400dc040000f6
:020000040000fa
:04022800dc040000f2
:020000040000fa
:04022c00dc040000ee
:020000040000fa
:04023000dc040000ea
:020000040000fa
:04023400dc040000e6
:020000040000fa
:04023800dc040000e2
:020000040000fa
:04023c00dc040000de
:020000040000fa
:04024000dc040000da
:020000040000fa
:04024400dc040000d6
:020000040000fa
:04024800dc040000d2
:020000040000fa
:04024c00dc040000ce
:020000040000fa
:04025000dc040000ca
:020000040000fa
:04025400dc040000c6
:020000040000fa
:04025800dc040000c2
:020000040000fa
:04025c00dc040000be
:020000040000fa
:04026000dc040000ba
:020000040000fa
:04026400dc040000b6
:020000040000fa
:04026800dc040000b2
:020000040000fa
:04026c00dc040000ae
:020000040000fa
:04027000dc040000aa
:020000040000fa
:04027400dc040000a6
:020000040000fa
:04027800dc040000a2
:020000040000fa
:04027c00dc0400009e
:020000040000fa
:04028000dc0400009a
:020000040000fa
:04028400dc04000096
:020000040000fa
:04028800dc04000092
:020000040000fa
:04028c00dc0400008e
:020000040000fa
:04029000dc0400008a
:020000040000fa
:04029400dc04000086
:020000040000fa
:04029800dc04000082
:020000040000fa
:04029c00dc0400007e
:020000040000fa
:0402a000dc0400007a
:020000040000fa
:0402a400dc04000076
:020000040000fa
:0402a800dc04000072
:020000040000fa
:0402ac00dc0400006e
:020000040000fa
:0402b000dc0400006a
:020000040000fa
:0402b400dc04000066
:020000040000fa
:0402b800dc04000062
:020000040000fa
:0402bc00dc0400005e
:020000040000fa
:0402c000dc0400005a
:020000040000fa
:0402c400dc04000056
:020000040000fa
:0402c800dc04000052
:020000040000fa
:0402cc00dc0400004e
:020000040000fa
:0402d000dc0400004a
:020000040000fa
:0402d400dc04000046
:020000040000fa
:0402d800dc04000042
:020000040000fa
:0402dc00dc0400003e
:020000040000fa
:0402e000dc0400003a
:020000040000fa
:0402e400dc04000036
:020000040000fa
:0402e800dc04000032
:020000040000fa
:0402ec00dc0400002e
:020000040000fa
:0402f000dc0400002a
:020000040000fa
:0402f400dc04000026
:020000040000fa
:0402f800dc04000022
:020000040000fa
:0402fc00dc0400001e
:020000040000fa
:04030000dc04000019
:020000040000fa
:04030400dc04000015
:020000040000fa
:04030800dc04000011
:020000040000fa
:04030c00dc0400000d
:020000040000fa
:04031000dc04000009
:020000040000fa
:04031400dc04000005
:020000040000fa
:04031800dc04000001
:020000040000fa
:04031c00dc040000fd
:020000040000fa
:04032000dc040000f9
:020000040000fa
:04032400dc040000f5
:020000040000fa
:04032800dc040000f1
:020000040000fa
:04032c00dc040000ed
:020000040000fa
:10040000cf6321000eff24000e01880000000000d1
:10041000000020000000e000020032000001200087
:100420002002880014000700650107000000e000ba
:1004300003003a00005a21000100200002003700aa
:100440000000200001002000810f70000100320038
:100450000f000700000020000000e0000200320052
:100460000000020000000000be4702000000000083
:100470000040da000000fe00000120000000e00063
:1004800002003200002020009001880000000600d9
:10049000a1028800800478000000eb001f003700f4
:1004a000e284440054a0b4009905ba00e2844400f8
:1004b00054a0b4009906ba00e284440054a0b400e9
:1004c0000006eb00476fde00fd07b200ae018800ba
:1004d000636ce10003003a000ad801000000eb0061
:1004e0000e003700606ce10008003a00004deb00a0
:1004f0000a05e800020039003420ec000af0a000f0
:100500008b05e900f9ff3e00040037006168e10057
:10051000010032000086eb000b00070019c7ba008b
:100520001905ba000e04e00003003a000a00e000da
:10053000dbff3a0000000600fe07b200ae028800b2
:100540008a047800f5ff37000cd0a300e20f4d00bd
:100550001c00390089027800354dba000a05e80010
:10056000020039003420ec000af0a0008b05e900fd
:100570000f003200254dba000a05e80002003900dc
:100580003420ec000af0a0008b05e90008003200de
:100590000c00e0000600320015cdba000a05e800a4
:1005a000020039003420ec000af0a0008b05e900bd
:1005b0008984e80054a0b4000b00e000e2ff3a0098
:1005c000000006009902ba00055d78008b05e9007d
:1005d000f7ff3200c82ade00055d78008b05e900d0
:1005e000f3ff32000c00e000f1ff320019ddba0029
:1005f000eeff370066480400000000005048040089
:1006000000000000ae250400000000008c32040051
:1006100000000000fa320400000000001233040061
:1006200000000000ca38040000000000ec260400ae
:100630000000000044390400000000005c390400a0
:10064000000000005046040000000000563f040077
:100650000000000012450400000000002c3e0400d1
:10066000000000005a3c0400000000006242040048
:10067000000000007a460400000000003a18040060
:10068000000000001438040000000000a82e040040
:10069000000000005444040000000000d63c0400a8
:1006a00000000000d4440400000000005a2a0400a6
:1006b00000000000be4804000000000024480400c0
:1006c00000000000a82f0400000000003a480400c9
:1006d000000000000e480400000000004447040031
:1006e00000000000ce46040000000000184904008d
:1006f000000000003600f800809fbe00829fbe0010
:10070000849fbe00869fbe000008200029220700ab
:100710004f03be004f02be004f01be004f00be009f
:100720003600f900004006003600f800809fbe0049
:10073000829fbe00849fbe00869fbe0000082000ee
:100740001c2207004f03be004f02be004f01be0037
:100750004f00be003600f900004006003600f800e9
:10076000809fbe00829fbe00849fbe00869fbe0009
:10077000000420000f2207004f03be004f02be00fe
:100780004f01be004f00be003600f90000400600d9
:100790003600f800809fbe00829fbe00849fbe008e
:1007a000869fbe0000022000022207004f03be0009
:1007b0004f02be004f01be004f00be003600f900e0
:1007c000004006003600f800809fbe00829fbe00f9
:1007d000849fbe00869fbe0010002000f521070008
:1007e0004f03be004f02be004f01be004f00be00cf
:1007f0003600f900004006003600f800809fbe0079
:10080000829fbe00849fbe00869fbe002000200005
:10081000e82107004f03be004f02be004f01be009b
:100820004f00be003600f900004006003600f80018
:10083000809fbe00829fbe00849fbe00869fbe0038
:1008400040002000db2107004f03be004f02be0026
:100850004f01be004f00be003600f9000040060008
:100860003600f800809fbe00829fbe00849fbe00bd
:10087000869fbe0080002000ce2107004f03be00ef
:100880004f02be004f01be004f00be003600f9000f
:10089000004006003600f8003200f8003400f8008e
:1008a00010002000a00188000020200000d0fe00e1
:1008b0000030a800418a8000108a800001000100f9
:1008c0002e63a800d063a8000b88a9003400f900ab
:1008d0003200f9003600f900004006003600f8004a
:1008e0000800fa0010002000c0bf9f008a34a80052
:1008f00062a4800073a4800061014100e08149008e
:1009000062a4880073a488000028a900d0bf9f00bb
:100910000000eb00e0bf9f00f0bf9f0062a48000da
:1009200073a48000f2bf9f00e0bf9f006fb89700e4
:100930001614e30012003600244121006fb897001e
:1009400000004000000042001000780020019000ec
:10095000b0019000ffb8970002814000e08149009b
:1009600022009800330098006fb897000000e8005c
:10097000e0bf9f006fb897001614e300efff3e0042
:100980008c34ef008e34ef000028a9005fb8970088
:1009900021002000010078005a0d0700cfb9970010
:1009a00003006000c0bf9f003676ef000080fa00b1
:1009b0003600f900004006000040da000000fe00aa
:1009c00000000500839f68000100e00002003d0078
:1009d00060001000e08018000300e00002003d000d
:1009e00060011100e0811900070007004f00e000de
:1009f00002003b0060001000e080180000000600cc
:100a00006011b800d2013700020250008382580002
:100a100061003900030371006200320005037200b7
:100a2000590032000300e0005500330017003a007f
:100a30000100e0004b0032000208e1000600310036
:100a4000050009004288d800010178008001eb0010
:100a50008000eb00000006006110e100550032004c
:100a60000002be00050009008280d80080027800e4
:100a700004007800050009004288d80001017800d0
:100a80008001eb008500780000000600889fbe0012
:100a90008a9fbe008c9fbe000386cf000c06e90033
:100aa0008c1f78008c19dd00f00216000512de00a4
:100ab000848171000c11dd000003be008004eb0096
:100ac000053cde008c3bdd000532de0084837300d4
:100ad0000c33dd000700780088007800050009006d
:100ae0004388d8000202b8000306b8008c82420096
:100af00060854e008005eb000402530085825b0098
:100b00000a055c008b855c000b0033008000eb0065
:100b10004f0678000c21de00700516000a2ddd005e
:100b20000a0171008c29de004f06be004f05be0091
:100b30004f04be00000006000202420083824a0009
:100b400060054d00e0854d000000e9000b00e0006d
:100b5000eeff3d000202420083824a000000e900ed
:100b6000eaff37000000e000120032000500090033
:100b70000280d800010178008000eb000000060030
:100b80000401be00010037006011b8001000200011
:100b90008000eb00000006000001be006000b8000d
:100ba000000006000001be00f0ff2f00f1ff2f0043
:100bb000000006006011b80000000600889fbe001b
:100bc0008a9fbe008c9fbe001b0020000202be0058
:100bd0000586680006002800060666004709de0054
:100be000f20fb200820032000243e80080003200bf
:100bf000c729de00f30fb2007d0032000343e80096
:100c00007b003200f107b2000170a000f507b200ce
:100c10000570a000c708dd004903de008680700073
:100c20004700dd00c72add004923de00868272000e
:100c30004722dd000305510004035000858358005e
:100c40000300310000004000818048000a05e900ef
:100c50008c1f78008a9fbe000400500085805800d9
:100c60000402420085824a00000040008180480062
:100c70000005eb000004be006033b8000406be00af
:100c80000d48e10056003100050009004dccd800a8
:100c90000c01b8000d02b8008481410060824a0056
:100ca0008283530003045c0084845c0060055d0063
:100cb0000a00e00025003a00800578000d40e100c0
:100cc000490031008800780007007800050009001d
:100cd0004d88d8000c01b8000d02b8008481410095
:100ce00060824a006003110083835b0004045c009f
:100cf000e0845c000900e00021003a004f01be00e2
:100d00000300e0002b003200e301600007067300df
:100d10008c81710001003200640070004200de002e
:100d20004e5edd000c007000c258de0001e0a00045
:100d3000b4000700cf017800818071004f06be002b
:100d40004f05be004f04be00000006008c83430028
:100d50000d044c00e0844c0060054d000000e900eb
:100d60000a00e000d4ff32008c8343000d044c00e5
:100d7000e0844c0060054d000000e900ceff370024
:100d80000c0343008d834b0060044c00e0844c0056
:100d90000000e9000900e000d8ff32000c03430026
:100da0008d834b0060044c00e0844c000000e9009f
:100db000d2ff37004200de004e5edd000c00700006
:100dc000c258de0001e0a000cf0178000300e0007f
:100dd000daff320060001000e0801800d7ff370013
:100de000f0ff2f00aaff3700f0ff2f00b9ff3700f8
:100df0000404be002b010700870678000004fd00f4
:100e00008104fd0027010700078366000678a30020
:100e1000030032000960a7000800be002c00370064
:100e20000d78a300020032000800be002800370041
:100e30000778a30026003a0001f0a10009f0a10004
:100e40000668a30003003200f1ff2700f0ff2f0027
:100e5000baff37000d68a300030032000800be008f
:100e60008c807000b5ff37000768a30007003a00c8
:100e70000648a30003003200f1ff2700f0ff2f0017
:100e8000aeff37000d48a300030032006000b80039
:100e90008c807000a9ff37000748a30004003200cf
:100ea00001f82700000020008c807000a3ff3700ad
:100eb000210007000004fd008104fd000205780008
:100ec0001d0007000802be008a01780059ff3700a4
:100ed0000160a00012022000d2b1880097ff370005
:100ee0000100e000120032000500e00010003200b6
:100ef000889fbe008a9fbe008c9fbe000006eb004c
:100f000001f8a3000300320060001000e080180028
:100f10000cf0a00005f8a3000300320060021200ec
:100f2000e0821a000cf0a2008005eb0041ff3700c0
:100f30006000b800020005004f0ade004709de002d
:100f4000f107b200f20fb2000b003200f207b1005d
:100f50000170a000c708dd00c901de0083807000b9
:100f60004700dd000400a60000000600600010003d
:100f7000e080180000000600810f700001003a00b8
:100f8000000006008182cf000500e00010003e0056
:100f90008082cf00ee8242007028e1000400390018
:100fa00007003e00800078000000eb000e003700d4
:100fb000708312008600de000500dd000a003700a5
:100fc000708352008600dd000000eb000600370051
:100fd000e28252008508dd00708312000603de0005
:100fe000868070000500dd007507b0000501ea008d
:100ff0000400a6000000060060001000e080180059
:101000000000060081017000270032008002eb0022
:1010100001f8a3000300320060001000e080180017
:1010200015002000f40720000202420020003400d6
:10103000f70320008703600006042000000363001c
:1010400002082000000161004700de00c909dd0040
:1010500000807100c708de000600e00008003200d2
:1010600087037100060032001000b0000180b0005c
:101070000188a30002003200c108de000402e8007b
:10108000f107b200f30f20000320e10003003d0050
:101090004722dd00810072002900370001f8270097
:1010a0000000eb00260037006000b80000000600da
:1010b000680212007f20e100020034006000b800e6
:1010c0001f0037006011b8007020e10004003500f7
:1010d00080017800010078008000eb00700252006f
:1010e0000400e00009003400f00312000719dd00dd
:1010f0008419de000703dd00868171000400de0034
:10110000070bdd00060070008408de00f7ff2700f3
:1011100083836300870371000600280003036300d4
:10112000070032000700e00003003a0061016000a0
:1011300002817300020032001000b0000180b00094
:101140000500a6000000060001f0a0000000060057
:10115000889fbe008a9fbe0000827000040271005a
:1011600004827100260032000004be000200be00ae
:101170006011b8006b092000950220000182cf00a9
:101180000a0039000541b1000082cf000700390094
:101190000541b1000982cf00040039000541b100ca
:1011a0000882cf00010039000541b100054252001c
:1011b000120032000a003b0082817100610164006c
:1011c0008100d1000080d3008984d3000884d3003b
:1011d0008b05e8000442e800f7ff3a0007003700fb
:1011e0000804440089844c000000480081804800c5
:1011f0008b05e9000442e900f9ff3a00030007000b
:101200004f05be004f04be00000006008100200014
:10121000618055000b003d000b00200061fe2f0097
:101220000100e1001d003400828171006101640051
:101230008904d1000884d3000000e800faff3a00d6
:101240007100200061006400030070000200600073
:101250000900320061044400e0844c000988a500c4
:10126000050032008b05e8006808e10002003a0042
:101270008904d1000884d300f20f20000258e10055
:1012800005003d00c75ddd00f907b20089807500eb
:1012900008007800000006000bf827008b0078009b
:1012a000000005002700200001f0a7001700200023
:1012b000470bde00f60fb200040032000643e800e0
:1012c0000a0032004702b300000006000103780064
:1012d000f607b2000603700002003a000703b300ed
:1012e000000006008702b30000000600010378003a
:1012f000f607b20006037000020032000770a0007b
:0c130000000006000760a00000000600ce
:020000040000fa
:10130c001e14000018140000121400002414000015
:10131c00221400001c1400001614000028140000f5
:020000040000fa
:10132c00e8874700889fbe008a9fbe008c9fbe0046
:10133c008e1f78001a002000eab79f007810f80082
:10134c003a11f900203d2000c089880080fc2f0054
:10135c00f0898800403d2000008a88008098200099
:10136c00e089880000232100108a8800e15a2200bd
:10137c00218a8800c1282300418a8800a12f2300dc
:10138c00318a880021312300518a8800218a80000b
:10139c0001000100108a800021c220002041900031
:1013ac000044eb0021409800c808de00304190005a
:1013bc0031409800108a80008048900008489800be
:1013cc009048900018489800108a8000c040900007
:1013dc0054c0b30044409800d0409000584098004e
:1013ec00108a8000e0409000f2c9b300624098007f
:1013fc00f0409000e1c4b30071409800108a800066
:10140c0005c22000f30f2000204b900025489800c7
:10141c00c82ade00304b900035489800108a8000b6
:10142c0080529000085098009052900018509800ec
:10143c00108a8000c04a900044489800504a90009e
:10144c0058489800108a8000604a900062489800c2
:10145c007049900071489800108a8000c1142100d6
:10146c000381600082bf9f00205190000ff1970014
:10147c0022509800c808de00f1b79f00b0509000d1
:10148c00efe8970031509800108a80008058900047
:10149c00085898009058900018589800108a8000ae
:1014ac00c050900048509800d05090005850980070
:1014bc00108a8000e050900080c4eb0069509800c6
:1014cc00f0509000fbc7b3007b509800108a80004e
:1014dc00011621002059900021589800c808de0000
:1014ec003059900031589800108a8000806090002c
:1014fc00086098009060900018609800108a800036
:10150c00c058900048589800d058900058589800ef
:10151c00108a8000e058900069589800f0589000ac
:10152c007b589800108a8000811321002061900064
:10153c0021609800c808de0030619000316098008e
:10154c00108a8000f189800000c9900001c89800c1
:10155c00c808de0010c9900011c89800108a8000dd
:10156c00018a800020c9900021c89800c808de00bc
:10157c0030c9900031c89800108a8000c0c8900013
:10158c0048c89800d0c8900058c89800108a8000ad
:10159c00e0c8900068c89800f0c8900078c898001f
:1015ac00108a80004e3520008306670080d09000a2
:1015bc000dd098004877de0090d090001ed0980097
:1015cc00108a8000a0d0900028d09800b0d0900055
:1015dc0038d09800108a8000c0d090004dd0980070
:1015ec00d0d090005ed09800108a8000e0d090009f
:1015fc0001ceb30061d09800f0d090007ad0980062
:10160c00108a80008104210000d9900001d8980034
:10161c00c808de0010d9900011d89800108a8000fc
:10162c004104210020d9900021d89800c808de0080
:10163c0030d9900031d89800108a8000a104210084
:10164c0040d9900041d89800c808de0050d99000cd
:10165c0051d89800108a8000c104210060d99000f4
:10166c0061d89800c808de0070d9900071d8980035
:10167c00108a8000a0c0900029c09800b0c09000d3
:10168c007ac0b3003ac09800108a800080c09000e5
:10169c00c1cfb30001c0980090c0900019c0980051
:1016ac00108a8000c0c090000cc8b3004cc09800d9
:1016bc00d0c0900058c09800108a8000e0c0900004
:1016cc0068c09800f0c0900078c09800108a800024
:1016dc0080e0900008e0980090e0900018e09800fe
:1016ec00108a8000a0e0900028e09800b0e0900004
:1016fc0038e09800108a8000c0e0900048e0980024
:10170c00d0e0900058e09800108a8000e0e0900053
:10171c0068e09800f0e0900078e09800108a800073
:10172c0080e8900008e8980090e8900018e898008d
:10173c00108a8000a0e8900028e89800b0e890009b
:10174c0038e89800108a8000c0e8900048e89800bb
:10175c00d0e8900058e89800108a8000e0e89000eb
:10176c0068e89800f0e8900078e89800108a80000b
:10177c0080f0900008f0980090f0900018f098001d
:10178c00108a8000a0f0900028f09800b0f0900033
:10179c0038f09800108a8000a28c2300830061002e
:1017ac0040f2900041f09800c810de0050f290001a
:1017bc0051f09800118a8000a02b21008301600059
:1017cc0061f29000e3f09800c801de0071f2900025
:1017dc00f3f09800118a800081f9900088f8980045
:1017ec0091f9900098f89800118a8000a1f9900066
:1017fc00a9f89800b1f99000bbf89800118a800004
:10180c00c1f99000c8f89800d1f99000d8f8980068
:10181c00118a8000e1f99000e8f89800f1f9900045
:10182c00f8f89800118a8000814191008840990055
:10183c009141910098409900118a8000a14191003a
:10184c00a8409900b1419100b8409900118a8000dc
:10185c00c1419100c8409900d1419100d8409900f4
:10186c00118a8000e1419100e8409900f14191001a
:10187c00f8409900118a8000914190000374a100f6
:10188c0093409800118a8000914190000354a1006c
:10189c0093409800118a8000914190000344a1006c
:1018ac0093409800118a8000914190000364a1003c
:1018bc0093409800118a80001104a100118a8000c5
:1018cc001114a100118a8000914190000334a100f1
:1018dc009340980001782000718a8800413d2000d7
:1018ec00618a8800810c2000918a8800015e2100a9
:1018fc00a18a880001b32000818a8800b08a880000
:10190c00c16e2200c18a8800e28a880041942300bb
:10191c00d18a8800c1952300f18a8800c18a800091
:10192c0001000100b08a8000e1c02000204190003d
:10193c0021409800c808de003041900031409800ea
:10194c00b08a8000804890000c4898009048900025
:10195c001a489800b08a8000c04090004a40980015
:10196c00d040900058409800b08a8000e040900031
:10197c0069409800f040900031c6b3007140980067
:10198c00b08a800002c12000a04990002248980033
:10199c004811de00b049900032489800b08a8000af
:1019ac00005190000c509800105190001a50980063
:1019bc00b08a8000404990004a48980050499000f5
:1019cc0058489800b08a8000604990006948980097
:1019dc007049900071489800b08a8000e134200072
:1019ec002051900021509800c808de003051900022
:1019fc0031509800b08a80008058900008589800a8
:101a0c009058900018589800b08a8000c0509000f0
:101a1c0048509800d050900058509800b08a8000e0
:101a2c00e050900069509800f05090007b50980066
:101a3c00b08a8000013f2000205990002158980066
:101a4c00c808de003059900031589800b08a8000e8
:101a5c00806090000860980090609000186098007a
:101a6c00b08a8000c058900048589800d058900018
:101a7c0058589800b08a8000e05890006958980037
:101a8c00f05890007b589800b08a8000a0609000bd
:101a9c000ff1970022609800b0609000efe897007b
:101aac0031609800b08a8000918a800000c9900053
:101abc0001c89800c808de0010c9900011c8980031
:101acc00b08a8000a18a800020c9900021c89800ab
:101adc00c808de0030c9900031c89800b08a800078
:101aec00918a800040c9900041c89800c808de0067
:101afc0050c9900051c89800b08a8000a18a80001b
:101b0c0060c9900061c89800c808de0070c99000d8
:101b1c0071c89800b08a800080d090000dd09800d9
:101b2c0090d090001ed09800b08a8000a0d0900079
:101b3c0001c3b30021d09800b0d09000b1c0b30065
:101b4c0031d09800b08a8000613f200040d19000d5
:101b5c0041d09800c808de0050d1900051d09800b8
:101b6c00b08a8000e0d0900001cfb30061d0980023
:101b7c00f0d09000a1c0b30071d09800b08a800062
:101b8c0080d8900008d8980090d8900018d8980069
:101b9c00b08a8000a0d8900028d89800b0d89000c7
:101bac0038d89800b08a8000c0d8900048d89800e7
:101bbc00d0d8900058d89800b08a8000e0d8900017
:101bcc0068d89800f0d8900078d89800b08a800037
:101bdc0080e0900008e0980090e0900018e09800f9
:101bec00b08a8000a0e0900028e09800b0e090005f
:101bfc0038e09800b08a8000c0e0900048e098007f
:101c0c00d0e0900058e09800b08a8000e0e09000ae
:101c1c0068e09800f0e0900078e09800b08a8000ce
:101c2c0080e8900008e8980090e8900018e8980088
:101c3c00b08a8000a0e8900028e89800b0e89000f6
:101c4c0038e89800b08a8000c0e8900048e8980016
:101c5c00d0e8900058e89800b08a8000e0e8900046
:101c6c0068e89800f0e8900078e89800b08a800066
:101c7c0080f0900008f0980090f0900018f0980018
:101c8c00b08a8000a0f0900028f09800b0f090008e
:101c9c0038f09800b08a8000c0f0900048f09800ae
:101cac00d0f0900058f09800b08a8000e0f09000de
:101cbc0068f09800f0f0900078f09800b08a8000fe
:101ccc00a0c0900028c09800b0c0900038c0980008
:101cdc00b08a800080c0900008c0980090c090002e
:101cec0018c09800b08a8000c0c0900048c098000e
:101cfc00d0c0900058c09800b08a8000e0c090001e
:101d0c0068c09800f0c0900078c09800b08a80003d
:101d1c0080f8900008f8980090f8900018f8980057
:101d2c00b08a8000a0f8900028f89800b0f89000d5
:101d3c0038f89800b08a8000c0f8900048f89800f5
:101d4c00d0f8900058f89800b18a800061f89000a3
:101d5c00e8f8980071f8900008407800f0f89800c6
:101d6c00b18a80000141910080409900114191009d
:101d7c0090409900b18a800021419100a0409900c7
:101d8c0031419100b0409900b18a800041419100ed
:101d9c00c040990051419100d0409900b18a800017
:101dac0061419100e040990071419100f04099002f
:101dbc00b08a8000904090000174a10011409800fe
:101dcc00b08a8000904090000154a100114098000e
:101ddc00b08a8000904090000144a100114098000e
:101dec00b08a8000904090000164a10011409800de
:101dfc00b08a80001004a100b08a80001014a100e9
:101e0c00b08a8000904090000134a10011409800ed
:101e1c0002162100c01421000900090030197800b5
:101e2c0000782000108b88000037b000208b8800d1
:101e3c006fb097004f0778004f06be004f05be00ed
:0c1e4c004f04be008f00b1000000060033
:020000040000fa
:101e58000800fa00889fbe008a9fbe0080047800b0
:101e680010002000000f78000000eb001007980019
:101e780010079800b91890001e009000808f50003d
:101e8800c60136004a0320001e0090008a80b9006f
:101e98000080440060989000200798001e00900081
:101ea8008a80b9000080440070989000300798003c
:101eb8003e009000000040004117210000804000d3
:101ec80010007800e04090008180fb00f041900015
:101ed800c819dd00838170001e0190008a91b90045
:101ee8008280440001a19000110020000209dd0059
:101ef8000281ea0003016100e0419000624098001d
:101f08004811de00f0419000724098006042900055
:101f18000482fb00f0419000c819dd0083017200c3
:101f28001e0190008a91b9000281440012a190001c
:101f38000209dd000281ea0003016100e04190002e
:101f4800624098004811de00f0419000724098000d
:101f5800204290000482fb00b0419000c819dd00c7
:101f6800830172001e0190008a91b9000281440029
:101f780002a190000209dd000281ea00030161006c
:101f8800a0419000224098004811de00b041900026
:101f980032409800204290000482fb00b04190003b
:101fa800c819dd00830172001e0190008a91b900f2
:101fb8000281440012a190000209dd000281ea00ba
:101fc80003016100a0419000224098004811de0002
:101fd800b041900032409800404a90000482fb00d3
:101fe800d0499000c819dd00830172001e019000dd
:101ff8008a91b9000281440002a190000209dd0023
:1020080002817100c0499000424898004811de00e2
:10201800d049900052489800c04990008381fb0045
:10202800504990004811dd00028171001e029000a5
:102038008aa2b9008481440093a190008308dd003e
:10204800810071004049900041489800c808de00ae
:1020580050499000514898002e0090000000e90077
:1020680000004000814c21000080400010047800ee
:102078001e0090008a80b90000804400609890009b
:102088006f03b000abfc2f008f8545004145210050
:102098001a000900b11d78006b03b100281b070066
:1020a8001e0f60001e0090008a80b9000080440066
:1020b800d0c09100e1c06000620020008208dd000d
:1020c800384090000064a10001407000304498003e
:1020d8001e0090008a80b9000080440060c0910012
:1020e80061406000710020000100dd009840780028
:1020f8000174a10000cc70001e0090008a80b90015
:102108000080440070a09000c8609000406498006f
:102118004800de00d8609000506498001e009000cf
:102128008a80b9000080440040a090008868900030
:10213800006c98004800de0098689000106c9800c9
:102148001e0090008a80b9000080440020a89000fa
:1021580088709000007498004800de009870900025
:10216800107498001e0090008a80b9000080440016
:1021780010a89000a8709000207498004800de0015
:10218800b8709000307498001e0090008a80b900e2
:102198000080440030a89000e8589000605c9800e7
:1021a8004800de00f8589000705c98001e0090000f
:1021b8008b0778000000e00021003a0039189000f1
:1021c800e10f50001e003600384090000034a00097
:1021d80030449800a840900000cfb30000c06000d1
:1021e80020449800a848900080cfb30080c06000c9
:1021f8003140b300214c98001e0190000201e80014
:102208008a91b90082804400d1a09000686990004a
:10221800616c9800c808de0078699000716c9800bd
:10222800b840900000c060000004a000304498004e
:10223800284890008041b300204c98007100370076
:102248001e0090000000e0002b003200b91890003a
:102258001e0090008100e900808f500026003600a3
:10226800384090000034a000304498001e009000d0
:102278000000e9008a80b90000804400e0989000de
:10228800efc060002841900000cfb300004061001b
:102298000140700020449800a848900080cfb30007
:1022a80080c060003140b300214c98001e019000ae
:1022b8000201e8008a91b90082804400d1a0900010
:1022c80068699000616c9800c808de007869900021
:1022d800716c9800b840900000c060003040b300b6
:1022e80030449800a848900070ceb30000c0600049
:1022f800204c9800430037001e0090000000e000ca
:1023080025003200b91890001e0090008100e900f5
:10231800808f500020003a00384090000034a1001f
:10232800304498001e0090000000e9008a80b9003f
:1023380000804400e0989000efc0600028419000c1
:1023480000cfb300004061000140700020449800b5
:10235800a848900080cfb30080c06000214c98004e
:10236800e86890008040eb00616c98007869900004
:10237800716c9800b840900000c060003040b30015
:1023880030449800a848900070ceb30000c06000a8
:10239800204c98001b00370039189000e10f5000be
:1023a80018003a00384090000034a10030449800ea
:1023b800a840900000cfb30000c0600020449800ff
:1023c800a848900080cfb30080c060003140b300bf
:1023d800214c9800e86890008040eb00616c980000
:1023e80078699000716c9800b840900000c0600057
:1023f8000004a00030449800284890008041b300b1
:10240800204c98001e0090008a80b900008044008b
:10241800c0a89000ffc06000320020008208dd00e4
:10242800384890006740600001407000304c9800c8
:102438001e0090008a80b90000804400d0a8900057
:10244800ffc060004849900000ceb3000040610022
:1024580001407000404c9800484090000034a000b3
:1024680040449800284090000064a0002044980050
:1024780029189000e10f500041003a0038489000b8
:102488000004a000304c9800484890000064a00068
:10249800404c98001e0090008a80b90000804400db
:1024a80030b09000a8689000206c98004800de00ca
:1024b800b8689000306c98001e0090008a80b900bf
:1024c8000080440040b09000c8689000406c9800bc
:1024d8004800de00d8689000506c98006850900062
:1024e8000040eb00605498007850900010c1b30091
:1024f800705498000858900090c1b300005c980090
:102508001858900030c0b300105c98001e0090006e
:102518008a80b9000080440090b09000ffc060003d
:102528006851900000ceb300004061000140700087
:10253800605498001e0090008a80b9000080440012
:1025480040c091000004e00007003200684090009d
:1025580080c0b300604498007840900000c3b30086
:1025680070449800060037006840900040c0b300ef
:10257800604498007840900000c3b300704498000d
:102588001e0090000000e80010079800b91890009d
:102598001e009000808f50003bfe3e0029189000de
:1025a800e10f500005003a00f71607001e0f600003
:1025b800090078009a0a07001e0f60001e007800c4
:1025c8004f05be004f04be000080fa000000060060
:020000040000fa
:1025d8000800fa006000b800c0bf9f00d1bf9f008c
:1025e8000000eb00e0bf9f00eca00a00840f000091
:1025f800f0bf9f000120210011a88800a10720003a
:1026080021a888007fb897000000e0000900320088
:102618007fb89700e60f5000060032007fb8970099
:10262800e10f5000030032007fb89700e70f500019
:102638002d003a0000202100a1072000c0bf9f0004
:10264800d1bf9f007fb89700e60f500013003200fb
:10265800627c800050820a00020000000281fb00b8
:102668008001eb0001eb2000819ab9000110b8004d
:10267800810042004fb99700dfb99700000141007f
:1026880081814900c2bf9f00d3bf9f004fba970006
:10269800dfba970014a8880025a888007fb897009b
:1026a800e70f50001e003a0098a00a00860f0000ad
:1026b800e0bf9f004fb99700dfb99700efb89700c8
:1026c8000202be00010378000603e900030033009c
:1026d8008582d1000482d300fbff3700c4bf9f006e
:1026e800d5bf9f000e0037007fb89700e50f500058
:1026f80005003a0000d0270001002000c0bf9f005d
:10270800d1bf9f00060037004fb99700dfb9970087
:102718000000eb00e00f5100e08f59000401320087
:102728004fb89700dfb8970050a8880061a88800c4
:102738007fb89700e10f5000030032007fb8970080
:10274800e30f500053003a000000eb0084afab00e9
:10275800f7003200307c80006f006000e0bf9f000f
:10276800efb897008100e9000000eb00e78f500008
:10277800ef003e004fb89700dfb897006fb9970099
:102788008001eb008df80700c0bf9f00d1bf9f00fc
:10279800f00f2000880fb600e0bf9f006fb99700c8
:1027a800630151000000eb00510c2000810f510023
:1027b800df003e006fb897004fb99700dfb9970068
:1027c8008000eb00809ab9000200b8008100420046
:1027d800c0bf9f00d1bf9f0098a00a008a0f0000c9
:1027e800e0bf9f00efb897000000eb00e38f5000b8
:1027f800cf003e006fb8970064001000e0bf9f0054
:102808004fb89700dfb897006fb997008001eb00c9
:102818006af80700f0a8880001a9880064a00a00e7
:102828008a0f0000e0bf9f00efb897008100e90021
:102838000000eb00e78f5000bd003e004fb8970046
:10284800dfb897006fb997008001eb005bf80700cd
:10285800c0bf9f00d1bf9f00507c80006700600010
:10286800e0bf9f00efb897008100e9000000eb008f
:10287800e78f5000ae003e004fb89700dfb89700d2
:102888006fb997008001eb004cf80700c0bf9f00ac
:10289800d1bf9f004fb99700dfb99700d2a8880031
:1028a800e3a888004fb89700dfb897008180d1006f
:1028b8000080d300c0bf9f00d1bf9f004fba9700d0
:1028c800dfba970074a8880085a888004fb89700d9
:1028d800dfb897008180d1000080d300c0bf9f007f
:1028e800d1bf9f004fb89700dfb89700b0a8880005
:1028f800c1a88800876fab000f003200dca00a0077
:10290800860f0000e0bf9f004fb99700dfb997001e
:10291800efb897000202be00010378000603e90041
:10292800030033008582d1000482d300fbff370007
:10293800c4bf9f00d5bf9f004fb89700dfb897006e
:1029480090a88800a1a8880090a88000a1a880006d
:1029580029f807000001be000000200001f823004c
:1029680094f8070030a9880041a98800b0a8800021
:10297800c1a8800020f807000001be000000200068
:1029880001f823008bf8070010a9880021a9880006
:102998008e0fe20061003d008f0fab000500320092
:1029a80012a8800023a88000c2bf9f00d3bf9f0049
:1029b8000400370034a8800045a88000c4bf9f00e9
:1029c800d5bf9f00707c80006f006000e0bf9f0053
:1029d800efb897008100e9000000eb00e78f500096
:1029e80053003e004fb89700dfb897006fb99700c3
:1029f8008001eb00f1f70700c0bf9f00d1bf9f0027
:102a0800f00f2000900fb600e0bf9f006fb997004d
:102a1800630151000000eb00510c2000810f5100b0
:102a280043003e006fb897004fb99700dfb9970091
:102a38008000eb00809ab9000200b80081004200d3
:102a4800c0bf9f00d1bf9f0098a00a00920f00004e
:102a5800e0bf9f00efb897000000eb00e38f500045
:102a680033003e006fb8970064001000e0bf9f007d
:102a78004fb89700dfb897006fb997008001eb0057
:102a8800cef7070070a9880081a9880064a00a0011
:102a9800920f0000e0bf9f00efb897008100e900a7
:102aa8000000eb00e78f500021003e004fb8970070
:102ab800dfb897006fb997008001eb00bff70700f8
:102ac800c0bf9f00d1bf9f00907c8000670060005e
:102ad800e0bf9f00efb897008100e9000000eb001d
:102ae800e78f500012003e004fb89700dfb89700fc
:102af8006fb997008001eb00b0f70700c0bf9f00d7
:102b0800d1bf9f004fb89700dfb8970050a9880041
:102b180061a9880010002000050037002a35ef0061
:102b28002c35ef002e35ef003035ef001000200077
:082b38000080fa000000060015
:020000040000fa
:102b400042130000840000008200000003820000a5
:102b500000421000ffff000000ffff000e053100e3
:102b6000005048006d05870013000000038100003d
:102b700000421000ffff000000ffff000b0f3100bc
:102b800000504800ad0e87001300000003810000d4
:102b900000461000ffff000000ffff003506310077
:102ba00000504800f4051f004e0000000001000026
:102bb00000401000ffff000000ffff000c081300a2
:102bc00000504800a9071f004e000000000100004f
:102bd00000441000ffff380010ffff003f00f3002b
:102be0000150480025001f004e00000042135a000b
:102bf000137213008a13a200130500007a15000057
:102c00001800000082000000030000000000000027
:102c1000ffff000000ffff000000000000000000b8
:102c200000000000000000001a1600000c00000068
:102c3000800000000010000074010000800000000f
:102c40002a14000060000000820000000300000061
:102c50000000000000000000000000000000000074
:102c60000000000000000000000000000000000064
:102c70000000000000000000000000000000000054
:102c8000000000008800000001000000003000008b
:102c900000190100400100000000000000000000d9
:102ca000000000000000000000000000000008001c
:102cb0000000000000000000000000000000000014
:102cc0000000000000000000000000002e160000c0
:102cd000040000008000000026160000080000002c
:102ce0008200000080000000005400008900000005
:102cf000f01500000e00000080000000fe1500002e
:102d00000e00000082000000504656003f124500b1
:102d10002c3e5a003c62420006000000d015000024
:102d200010000000820000007a463a0018143800b3
:102d3000a82e540044d63c00d444070000000000f4
:102d40003216000004000000820000005a2a010030
:102d500000000000e01500001000000080000000ee
:102d6000321500002600000082000000020003006f
:102d7000000200000300c400510000003dee00000e
:102d800000c476000000bf0000000000fc890000c5
:102d900000030000ffff030000725b00ffff000064
:102da0002e1200008a00000080000000a81500001c
:102db0001400000080000000005000000a00000025
:102dc0008000000058150000220000008200000072
:102dd00002000300000200000300e60041000000c2
:102de0001bfe0000000352000000ff000400000072
:102df000fdb2000000040000ffff0400000000001e
:102e0000b81200008a00000080000000bc1500001d
:102e100014000000800000000a5000000a000000ba
:102e20008000000074110000ba0000008200000061
:102e3000000e1c000e380e000000110011000000f2
:102e40000000000000000000000000000000000082
:102e50000000000000000000000001000000000071
:102e6000000002000000000000000300000000005d
:102e7000000003000000000001000000002000002e
:102e800001000100002100000100020000220000fa
:102e900001000300002300000100040000240000e2
:102ea00001000500002500000100060000260000ca
:102eb00001000700002700000100080000280000b2
:102ec000010009000029000001000a00002a00009a
:102ed00001000b00002b000001000c00002c000082
:102ee00001000d00002d000001000e00002e00006a
:102ef00001000f00002f0000020000000030000061
:102f00000200010000310000020002000032000057
:102f1000020003000033000002000400003400003f
:102f20000200050000350000c81400003a0000004f
:102f3000820000002a03600003960300cc03020015
:102f4000043804006e04a400040300000000000024
:102f50000000000000000000000000000000000071
:102f60000000000000000000000000000000000061
:102f70000000000000000000000000000000000051
:102f8000000000000c1600000e000000820000008f
:102f9000880c98000ca80c00800000000055000070
:102fa0008a000000021500003000000080000000d0
:102fb000c6130000640000008200000000800200d0
:102fc0000000000000000000000000000000000001
:102fd00000be48002448a8002f3a48000000000026
:102fe00000000000000000000000000000000000e1
:102ff000800200000000000000000000000000004f
:10300000000000000e48440047ce4600184900006a
:1030100000000000000000000000000000000000b0
:1030200000c61300ec13020000c61300ec130200ec
:1030300000c61300ec13020000c61300ec130200dc
:10304000000000008a1400003e0000008000000024
:103050003616000004000000820000000100040099
:10306000000000003a16000002000000800000008e
:04307000000000005c
:020000040000fa
:103074002000fa00881f7800000478001000200067
:10308400f0af9f000001eb0082b79f006000b80022
:1030940090b79f00a1b79f00b0b79f00c1b79f0032
:1030a400d0b79f00e1b79f00f0b79f0081bf9f009a
:1030b40090bf9f00a1bf9f00b0bf9f00c1bf9f00f2
:1030c400d0bf9f00e1bf9f001870a0004818900077
:1030d400401c990042149800720c9800182091002a
:1030e40081022000888040002061900021609800c7
:1030f400c808de003061900031609800a82090007c
:1031040041149800c810900068109000808f5000ff
:103114000200310068129000441498005810900086
:103124000000e00002003a00100020005014980053
:10313400081090000000e00002003a001000200097
:10314400001498009820900018309000808f500050
:1031540075003200a820900048389000808f5000fd
:1031640071003200a838900028219000483890005f
:10317400000051000100b80090b79f00a1b79f0064
:103184001fb19700afb19700b8389000f0801000dd
:103194000202be00010378000603e90003003300c5
:1031a4008502d1000482d300fbff370094b79f004f
:1031b400a5b79f00f82890001821900018309000bf
:1031c400000051000100b800b0b79f00c1b79f00d4
:1031d4003fb19700cfb1970088309000f080100085
:1031e4000202be00010378000603e9000300330075
:1031f4008502d1000482d300fbff3700b4b79f00df
:10320400c5b79f001fb19700afb197003fb09700bb
:10321400cfb09700800f5100818f59000400360011
:103224003fb09700cfb0970090b79f00a1b79f0021
:10323400481890008000eb00f0b79f0081bf9f000a
:1032440048a090008000eb00d0bf9f00e1bf9f002a
:103254003fb09700cfb09700e00f5000e08f5800c8
:10326400210032005fb99700efb997001fb09700b3
:10327400afb097000200b800d0b79f00e1b79f003d
:103284003fb19700cfb197005fb29700efb29700bc
:103294000500090042aad8008000eb00d0b79f00c7
:1032a400e1b79f005fb99700efb997007fb097002f
:1032b4008fb897000200b80090bf9f00a1bf9f0085
:1032c4003fb19700cfb197001fba9700afba9700ec
:1032d4000500090042aad8008000eb0090bf9f00bf
:1032e400a1bf9f002c0037000fb1970040032000be
:1032f4008091b9008200440071a190008001eb002c
:10330400d2b79f00e3b79f008fb097008088b900c1
:103314000000440070a090008000eb0090bf9f006c
:10332400a1bf9f001c0037000000eb0080b79f0086
:10333400b81890000fb09700808f50001600360028
:10334400400320000fb197008091b900820044002f
:1033540071a190008001eb00d2b79f00e3b79f00fa
:103364000fb197008091b9008200440071a19000d0
:103374008001eb0092bf9f00a3bf9f008fb0970016
:103384008100e80081b79f00381990008fb0970042
:10339400810f5100ebff3e0028189000e10f500010
:1033a4000f00320003003900e20f50006e003a00b3
:1033b400160037005fb09700efb0970080007800e8
:1033c400080078006e0007007faa970004006000e0
:1033d400f0af9f0010002000f0af9f0064003700a2
:1033e4005fb09700efb09700800078000800780085
:1033f40063000700ffaa970005006000f0af9f007c
:1034040010002000f0af9f0059003700581b9000b7
:1034140006249900182091008820910020c990006a
:1034240021c89800c808de0030c9900031c898004f
:103434005fb09700efb09700800078000800780034
:103444004f000700ffa8970001006000f0af9f0045
:10345400686890000004e000400032000818900002
:103464001fb19700afb197008000eb00020050003d
:1034740083805800f0b79f0081bf9f007fb0970002
:103484008fb89700581190007fb097008fb89700bd
:103494006102b8000500090042aad8008000eb00d0
:1034a400f0b79f0081bf9f001fb99700afb9970085
:1034b4005fb09700efb09700000051008180590081
:1034c400b0bf9f00c1bf9f003fb89700cfb897001f
:1034d400e00f5000e08f580004003a001000200074
:1034e40001002000b0bf9f00c1bf9f007fb19700c3
:1034f4008fb997003fb89700cfb897006102b80022
:103504000500090042aad8008000eb00b0bf9f006c
:10351400c1bf9f003fb89700cfb897008100d1008a
:103524000080d300b0bf9f00c1bf9f003fb8970089
:10353400cfb89700e00f5000e08f580004003a0025
:103544001000200001002000b0bf9f00c1bf9f00f9
:103554003fb89700cfb89700101c980010002000c7
:10356400f0af9f00020037000002eb00f4af9f00b1
:103574007fa897004f0478000080fa00000006003e
:020000040000fa
:103584000600fa00889fbe0000047800d1bf9f00a7
:1035940010002000b0bf9f000000eb00c0bf9f00e0
:1035a40028189000e10f5000630032000300390036
:1035b400e20f500027013a0082003700f81891000a
:1035c4005fb89700808f5000030036007818910090
:1035d400d0bf9f0006003700882091005fb8970095
:1035e400808f50000200310088209100d1bf9f00dd
:1035f400d82191005fb99700182091008000eb005a
:103604000300010018209100a05090008180fb006d
:10361400305090004800dd00008070001c00320033
:1036240018209100a05890008180fb003058900031
:103634004800dd0000807000150032001820910061
:10364400104078000028a3001100320018209100d7
:10365400a05090008180fb00305090004800dd00b5
:1036640000807000dfb897000108780018209100ee
:10367400a05890008180fb00305890004800dd0085
:1036840000807000dfb8970001087800ea00370076
:1036940018209100a05090008180fb0030509000d1
:1036a4004800dd00008070000d00320018209100f9
:1036b400104090000048a30009003a00182091002f
:1036c400a05090008180fb00305090004800dd0045
:1036d40000807000dfb8970001087800d60037003a
:1036e40018209100a05890008180fb003058900071
:1036f4004800dd00808070000000eb00da0032003a
:1037040018209100904090000000eb000148a300b5
:10371400d500320018209100a05890008180fb0051
:10372400305890004800dd0000807000dfb897003a
:1037340001087800c0003700cfb89700400320008c
:103744008088b90000004400e0b090000000eb0065
:103754000100e000c4003200b8209100182091005c
:10376400010001000000eb00c0bf9f00b8189000ea
:103774004fb89700808f5000af0036004003200000
:103784004fb997008091b90082004400e1b09000e5
:103794004fb997008091b9000201440072b19000c2
:1037a40082087800cfb897008100e800c1bf9f006d
:1037b40038199000cfb89700810f5100f0ff3e00f8
:1037c4009d0037000000eb00c0bf9f00b8189000b8
:1037d4004fb89700808f5000970036008004eb00ac
:1037e4004fb89700f400b9000000440090289100fd
:1037f4005fb89700808f5000060036004fb89700de
:10380400f400b9000000440010289100d0bf9f00cc
:103814000c0037004fb89700f400b90000004400d2
:10382400a02891005fb89700808f500005003100f8
:103834004fb89700f400b90000004400202891001c
:10384400d0bf9f004fb89700f400b90000004400b7
:10385400f02991005fb997004fb89700f400b900c0
:103864000000440030289100890078000300010022
:103874004fb89700f400b9000000440030289100cc
:10388400a05090008180fb00305090004800dd0083
:1038940000807000280032004fb89700f400b9008f
:1038a4000000440030289100a05890008180fb0063
:1038b400305890004800dd00008070001e00320087
:1038c4004fb89700f400b90000004400302891007c
:1038d400104078000028a300170032004fb897006a
:1038e400f400b9000000440030289100a05090007a
:1038f4008180fb00305090004800dd0000807000a3
:10390400dfb89700010878004fb89700f400b900b9
:103914000000440030289100a05890008180fb00f2
:10392400305890004800dd0000807000dfb8970038
:1039340001087800390037004fb89700f400b90047
:103944000000440030289100a05090008180fb00ca
:10395400305090004800dd000080700013003200f9
:103964004fb89700f400b9000000440030289100db
:10397400104090000048a3000c003a004fb8970094
:10398400f400b9000000440030289100a0509000d9
:103994008180fb00305090004800dd000080700002
:1039a400dfb89700010878001c0037004fb8970073
:1039b400f400b9000000440030289100a0589000a1
:1039c4008180fb00305890004800dd0000807000ca
:1039d400220032004fb89700f400b9000000440000
:1039e40030289100104090000048a3001d003200d0
:1039f4004fb89700f400b90000004400302891004b
:103a0400a05890008180fb00305890004800dd00f1
:103a140000807000dfb89700010878004fb8970065
:103a24000000e800c0bf9f00b81890004fb897008e
:103a3400808f50006aff3e00080078000f130700d3
:103a4400bfb8970001006000b0bf9f003fb8970067
:103a5400050037000000eb00030037000000eb0016
:103a6400010037000000eb004f04be000080fa00a4
:043a74000000060048
:020000040000fa
:103a78000600fa00881f7800000478001000200073
:103a8800c0bf9f000000eb00d0bf9f00e0bf9f00b9
:103a980018209100904090000174a10011409800f6
:103aa800b8209100182091000100010078189100b9
:103ab800e0bf9f0018209100a05090008180fb007b
:103ac800305090004800dd00008070001c0032007b
:103ad80018209100a05890008180fb003058900079
:103ae8004800dd00008070001500320018209100a9
:103af800104078000028a30011003200182091001f
:103b0800a05090008180fb00305090004800dd00fc
:103b180000807000efb89700010878001820910025
:103b2800a05890008180fb00305890004800dd00cc
:103b380000807000efb8970001087800290037006e
:103b480018209100a05090008180fb003050900018
:103b58004800dd00008070000d0032001820910040
:103b6800104090000048a30009003a001820910076
:103b7800a05090008180fb00305090004800dd008c
:103b880000807000efb89700010878001500370032
:103b980018209100205990000281fb00b058900035
:103ba800c808dd00810071000000eb00d000320081
:103bb80018209100904090000000eb000148a300fd
:103bc800cb00320018209100a05890008180fb00a3
:103bd800305890004800dd0000807000efb8970072
:103be8000108780028189000e10f50000400320006
:103bf800b3003900e20f5000b8003a002300370044
:103c0800dfb89700400320008088b9000000440016
:103c1800e0b090000000eb000100e000b4003200ca
:103c2800b820910018209100010001000000eb006d
:103c3800d0bf9f00b81890005fb89700808f5000e1
:103c48009f003600400320005fb997008091b900bb
:103c580082004400e1b090005fb997008091b900fc
:103c68000201440072b1900082087800dfb8970022
:103c78008100e800d1bf9f0038199000dfb8970095
:103c8800810f5100f0ff3e008d0037005fb89700ac
:103c9800f400b900000044003028910090409000e2
:103ca8000174a100114098000000eb00d0bf9f00f4
:103cb800b81890005fb89700808f500080003600d9
:103cc8005fb89700f400b90000004400d0289100c4
:103cd8005fb89700f400b900000044003028910054
:103ce800010001005fb89700f400b900000044002b
:103cf80010289100e0bf9f005fb89700f400b9005a
:103d08000000440030289100a05090008180fb0002
:103d1800305090004800dd0000807000280032001c
:103d28005fb89700f400b900000044003028910003
:103d3800a05890008180fb00305890004800dd00ba
:103d4800008070001e0032005fb89700f400b900d0
:103d58000000440030289100104078000028a3009b
:103d6800170032005fb89700f400b9000000440063
:103d780030289100a05090008180fb0030509000c6
:103d88004800dd0000807000efb897000108780057
:103d98005fb89700f400b900000044003028910093
:103da800a05890008180fb00305890004800dd004a
:103db80000807000efb897000108780039003700dc
:103dc8005fb89700f400b900000044003028910063
:103dd800a05090008180fb00305090004800dd002a
:103de80000807000130032005fb89700f400b9003b
:103df8000000440030289100104090000048a300c3
:103e08000c003a005fb89700f400b90000004400c5
:103e180030289100a05090008180fb003050900025
:103e28004800dd0000807000efb8970001087800b6
:103e38001c0037005fb89700f400b9000000440088
:103e480030289100a05890008180fb0030589000e5
:103e58004800dd0000807000220032005fb8970043
:103e6800f400b90000004400302891001040900090
:103e78000048a3001d0032005fb89700f400b900a5
:103e88000000440030289100a05890008180fb0079
:103e9800305890004800dd0000807000efb89700af
:103ea800010878005fb897000000e800d0bf9f00c5
:103eb800b81890005fb89700808f500080ff3e00d0
:103ec80008007800ec110700cfb8970001006000e7
:103ed800c0bf9f004fb89700050037000000eb00f7
:103ee800030037000000eb00010037000000eb0082
:0c3ef8004f0478000080fa000000060073
:020000040000fa
:103f04001800fa00889fbe008a1f78008104780098
:103f14001100200091b79f006011b800a2b79f0064
:103f2400b3b79f008000eb00c1b79f00d1b79f00db
:103f3400e1b79f00e1ef9f0082bf9f0093bf9f0006
:103f4400ec01b900c14921008100410091007800d1
:103f5400d1b79f0021002000e1b79f00818f54005a
:103f640002003a008a34a80003003700e18f5400ad
:103f740001003a008a14a8008000eb00c1b79f003a
:103f84004fb19700dfb09700810f5100d700310087
:103f940000054000ec00b900814921000104400003
:103fa4000900e00003003a0010c0b300e0ef9f00f6
:103fb40036003700980078004fb0970000004000aa
:103fc40000804000100078001000e0002d003d004b
:103fd400980078004fb09700000040000080400037
:103fe4001000780010009000890f500022003a0061
:103ff400980078004fb09700000040000080400017
:104004001000780040019000d001900098007800e2
:104014004fb097000000400000804000100078007e
:10402400f000900060009000000041008180490091
:1040340080bf9f0091bf9f00980078004fb0970009
:104044000000400000804000100078002002900032
:10405400b00290000fb997009fb9970010c0b30049
:10406400820f5200838f5a0001003d000040eb0094
:10407400e0ef9f00050037000040eb00e0ef9f00f9
:10408400020037000040eb00e0ef9f006fe897006c
:104094000004e0008e003200980078004fb09700d2
:1040a40000004000008040001000780070014000d3
:1040b4000a014100980078004fb0970000004000ca
:1040c4000080400010007800e4004000980178006f
:1040d4004fb09700000040000080410010007800bd
:1040e4001070a000120078007c8157004a0a070073
:1040f40090b79f00980078004fb0970000004000f0
:1041040000804000100078009fb0970001f0a700e5
:104114008100ea008100ea00cf08de0000010a0005
:1041240010000000980078004fb097000000400095
:1041340000804000100078001070a1000028ab003f
:104144002a00320060a4800071a4800011a20a0039
:104154000008000000004100e080480060a48800de
:1041640071a4880010002000a0bf9f000000eb0095
:10417400b0bf9f00c0bf9f0062a4800073a48000f2
:10418400c2bf9f00b0bf9f003fb897001614e30062
:1041940012003600244121003fb89700000040007f
:1041a400000042001000780020019000b00190004f
:1041b400cfb8970002814000e081490022009800b6
:1041c400330098003fb897000000e800b0bf9f009c
:1041d4003fb897001614e300efff3e008c34ef0065
:1041e4008e34ef000028a9002fb8970098007800bb
:1041f4004fb097000000400000804000100078009d
:1042040020019000b001900082bf9f0093bf9f00e7
:104214000fb997009fb99700980078004fb09700a6
:10422400000040000080400010007800f000900082
:1042340060009000000051008180590080bf9f0001
:1042440091bf9f000fb997009fb99700980078001d
:104254004fb097000000400000804000100078003c
:10426400d00090004000900000005100818059006f
:1042740080bf9f0091bf9f00980078004fb09700c7
:10428400000040000080400010007800f000900022
:10429400600090000fb997009fb99700020040009a
:1042a4008380480080bf9f0091bf9f0098007800e2
:1042b4004fb09700000040000080400010007800dc
:1042c4000fb997009fb99700220098003300980017
:1042d4004fb097000000e800c0b79f00cfb0970030
:1042e4005fb09700808f50002dff39001fb09700fa
:1042f4004f0578004f04be000080fa00000006005d
:020000040000fa
:104304000400fa008002780011002000e1bf9f0041
:104314001504e000b6003200f5409000efcf5000e5
:1043240016003e0065499000f54090000281fb00b4
:104334008180fb008110dd0001007800d02bb700e4
:1043440035499000f54090000281fb008180fb001c
:104354008110dd0001007800f02bb70025499000a2
:10436400f54090000281fb008180fb008110dd009c
:1043740001007800202bb7001c0037007541900025
:104384008000eb00ff4f51009a003e006549900009
:10439400f54090000281fb008180fb00f08050001a
:1043a4008110dd0001007800d22bb7003549900060
:1043b400f54090000281fb008180fb00f0805000fa
:1043c4008110dd0001007800f22bb7002549900030
:1043d400f54090000281fb008180fb00f0805000da
:1043e4008110dd0001007800222bb700f540900019
:1043f400e7cf500004003e00f540900081c040002b
:10440400e1ff9f0018003700f5409000efcf500007
:1044140005003e00f5409000e8c0500081c0400017
:10442400e1ff9f0010003700f5409000f7cf5000e7
:1044340005003e00f5409000f0c0500081c04000ef
:10444400e1ff9f0008003700754190008000eb00f9
:10445400ff4f510067003e00f5409000f8c0500047
:1044640081c04000e1ff9f00f540900001b12000b1
:1044740091417800554a90006ff997000482fb003f
:104484000281fb000221dd0082c8710091417800a5
:10449400454a90006ff997000482fb000281fb00fb
:1044a4000201e8000221dd0082c87100f54090009d
:1044b4008180fb0002b820008280400015489000f3
:1044c40080487800854890000104e0000b00320029
:1044d400e5409000e6cf500008003e0005499000fa
:1044e400e54090000281fb008180fb008180400058
:1044f4008110dd00010078000e2bb700e54090002c
:10450400e3cf50001d00320004003e00e1cf500014
:104514000e00320013003e0006003700e5cf5000c5
:10452400220032001b003900e6cf50002b003a0075
:10453400240037002e16a800454890000004e0002f
:104544002b0032003016a800290037002e36a800b0
:10455400454890000004e000250032003036a800f1
:10456400230037002e56a800454890000004e000c0
:104574001f0032003056a8001d0037002e76a80018
:10458400454890000004e000190032003076a8008d
:10459400170037002e96a800454890000004e0005c
:1045a400130032003096a800110037002eb6a80080
:1045b400454890000004e0000d00320030b6a80029
:1045c4000b0037002ed6a800454890000004e000f8
:1045d4000700320030d6a800050037002ef6a800e8
:1045e400454890000004e0000100320030f6a800c5
:1045f400efb89700010078000080fa000000060080
:020000040000fa
:104604000400fa0011002000e1bf9f008000eb00cd
:10461400f1bf9f000000e000a200320020019000e2
:104624000200e0009f003200a00090001101780019
:10463400b000900081006100f1bf9f00c0009000b5
:104644000100e00009003200c000900091017800f0
:10465400d00090007fb997008180610081005100f3
:1046640001f0a7008100ea00f1bf9f00a8810a00c1
:1046740010000000e38f50002400320005003c00cd
:10468400e18f500009003200e28f500084003a00ac
:1046940012003700e58f5000340032002700350047
:1046a400e68f50007e003a003c0037006001900025
:1046b400ffb89700810f5100020031001010a000d4
:1046c4004100370010099000ffb89700810f510096
:1046d4003d0036001010a1003b003700600190003f
:1046e400ffb89700810f5100020036001010a0009f
:1046f4003500370010099000ffb89700810f510072
:10470400310031001010a1002f003700600190002b
:10471400ffb89700810f510002003a001010a0006a
:104724002900370060019000ffb89700810f510005
:10473400250032001010a100230037006001900012
:10474400ffb89700810f5100020032001010a00042
:104754001d00370060019000ffb89700810f5100e1
:1047640019003a001010a10017003700100990003a
:10477400ffb89700810f51000600310060019000de
:10478400ffb89700810f5100020036001010a000fe
:104794000d0037001010a1000b0037001009900025
:1047a400ffb89700810f510004003e0060019000a3
:1047b400ffb89700810f5100020031001010a000d3
:1047c400010037001010a1001018a30017003200d8
:1047d40010017800e10061000104e00013003a00d8
:1047e4001000e00011003d00900090008100e800fe
:1047f4001100980010019000f0009000810f51000a
:10480400250039001000a000f0009000110098006d
:10481400800890000100e0001f00320000089000b2
:1048240000000100e0bf9f001b003700100178006a
:10483400e10061000104e000020032001018a3004e
:10484400020032001000e0001100350090009000da
:104854008100e8001100980010019000a008900069
:10486400810f51000c0039001000a100a008900035
:1048740011009800b00890000100e000060032002a
:104884003008900000000100e0bf9f0002003700e4
:104894008000eb0011009800efb89700010037008a
:1048a4008000eb00010078000080fa0000000600a0
:020000040000fa
:1048b4001400fa0080bf9f0091bf9f00a2bf9f0019
:1048c400b3bf9f00c4bf9f00d5bf9f00e6bf9f003a
:1048d400f7bf9f000000eb00e0b79f00f0b79f0018
:1048e40000002700840fb60023003200a109200035
:1048f4000001eb008007200053f820008049780075
:104904008149780082497800e2072000207c8000f9
:10491400000161000200a000710520006004200075
:1049240043f8200080497800814978008249780062
:10493400f2342c00eca10a00840f0000a8a00a00a5
:10494400840f000080cf5000050032007fb0970034
:104954008000e800f1b79f00820f5000f5ff360099
:10496400ffb09700f0342c00808f50000200360016
:1049740040002000e0b79f00eca10a00840f000073
:104984000fb897008180fb00808f50004b003200ed
:1049940084efab0049003a007fb8970063006000e1
:1049a4004800dd00f1cf2f00527c8000828060003f
:1049b40081007000517c88003fb8970050200a00a5
:1049c400860f00004fb89700b0200a00880f00003f
:1049d4005fb89700670060004400dd00f1f82f0025
:1049e400527c80008280600081007000517c8800cd
:1049f4006fb8970020200a008a0f00000fb99700b3
:104a0400a10920008007200053f820008049780085
:104a14008149780082497800eca10a00840f0000e3
:104a2400a8a00a00840f000080cf50002d0032009f
:104a3400e2072000207c8000000161000200a00049
:104a4400710520006004200043f8200080497800ac
:104a54008149780082497800f2342c00eca10a00e4
:104a6400840f0000a8a00a00840f000080cf50002b
:104a7400050032007fb097008000e800f1b79f0086
:104a8400820f5000f5ff3600eca10a00840f0000ed
:104a9400a8a00a00840f000080cf500004003a0050
:104aa400ffb09700f0342c00808f50000d003600ca
:104ab40020002000e0b79f000a003700eca10a00a4
:104ac400840f00000fb897008180fb00808f500096
:104ad4000400320084efab000200320080002000aa
:104ae400e0b79f0084efa80002022000f3342c00fa
:104af400217c80000100610005003a007fb097002e
:104b04008000e800f1b79f00830f5000f8ff3600e3
:104b140084afab0004003200ffb09700f0342c00e7
:104b2400808f50000200360000012000e0b79f0093
:104b34006fb197000200e00004003a0033a00a00bd
:104b4400840f000061001000010037006fb097006f
:084b54000080fa0000000600d9
:020000040000fa
:104b5c000200fa00881f7800000478000000eb00c7
:104b6c00e0bf9f00f0000a0018000000815a2100ed
:104b7c004861900041649800c808de0058619000bc
:104b8c0051649800015b2100686190006164980099
:104b9c00c808de007861900071649800010025005f
:104bac0008699000016c9800c808de001869900034
:104bbc00116c98004100250028699000216c980028
:104bcc00c808de0038699000316c980081aa80001a
:104bdc006871900061749800c808de0078719000cc
:104bec007174980091aa800008799000017c98005b
:104bfc00c808de0018799000117c98007191800033
:104c0c0028799000217c9800c808de003879900043
:104c1c00317c980071aa8000487190004174980012
:104c2c00c808de00587190005174980091a980005a
:104c3c0048699000416c9800c808de0058699000e3
:104c4c00516c9800a1a9800068699000616c980073
:104c5c00c808de0078699000716c9800b1a98000da
:104c6c000871900001749800c808de00187190005b
:104c7c0011749800c1a980002871900021749800cb
:104c8c00c808de003871900031749800e0bf9f00b6
:104c9c00c86890008180fb00586890004800dd00d7
:104cac0000807000efb89700810f5000150036009f
:104cbc00a3532100825a21006fb89700efb89700d8
:104ccc00c208dd00818041004200dd00000041008f
:104cdc0031187800211078006fb897000000e800b8
:104cec00e0bf9f00c86890008180fb00586890006e
:104cfc004800dd0000807000efb89700810f500075
:104d0c00edff3e000000eb00e0bf9f00e868900064
:104d1c008180fb00786890004800dd000080700006
:104d2c00efb89700810f5000160036002354210075
:104d3c00825a21006fb89700efb89700c208dd00c7
:104d4c00818041000080e8004200dd00000041004d
:104d5c0031187800211078006fb897000000e80037
:104d6c00e0bf9f00e86890008180fb0078689000ad
:104d7c004800dd0000807000efb89700810f5000f4
:104d8c00ecff3e000023210017060700a0aa8000bc
:104d9c00e8789000607c98004800de00f87890007d
:104dac00707c9800b0aa8000c8789000407c980075
:104dbc004800de00d8789000507c9800100020004d
:0c4dcc004f0478000080fa000000060090
:020000040000fa
:104dd8000200fa00881f7800000478000000eb0049
:104de800e0bf9f00f0000a0018000000c15b21002e
:104df8004861900041649800c808de00586190003e
:104e080051649800415c21006861900061649800d9
:104e1800c808de007861900071649800a100250040
:104e280008699000016c9800c808de0018699000b5
:104e3800116c9800e100250028699000216c980009
:104e4800c808de0038699000316c9800b1ab80006a
:104e58006871900061749800c808de00787190004d
:104e680071749800c1ab800008799000017c9800ab
:104e7800c808de0018799000117c9800c195800060
:104e880028799000217c9800c808de0038799000c5
:104e9800317c9800a1ab8000487190004174980063
:104ea800c808de005871900051749800c1aa8000ab
:104eb80048699000416c9800c808de005869900065
:104ec800516c9800d1aa800068699000616c9800c4
:104ed800c808de0078699000716c9800e1aa80002b
:104ee8000871900001749800c808de0018719000dd
:104ef80011749800f1aa800028719000217498001c
:104f0800c808de003871900031749800e0bf9f0037
:104f1800c86890008180fb00586890004800dd0058
:104f280000807000efb89700810f50001500360020
:104f380003562100c25b21006fb89700efb89700b5
:104f4800c208dd00818041004200dd000000410010
:104f580031187800211078006fb897000000e80039
:104f6800e0bf9f00c86890008180fb0058689000ef
:104f78004800dd0000807000efb89700810f5000f6
:104f8800edff3e000000eb00e0bf9f00e8689000e6
:104f98008180fb00786890004800dd000080700088
:104fa800efb89700810f5000160036008356210095
:104fb800c25b21006fb89700efb89700c208dd0008
:104fc800818041000080e8004200dd0000004100cf
:104fd80031187800211078006fb897000000e800b9
:104fe800e0bf9f00e86890008180fb00786890002f
:104ff8004800dd0000807000efb89700810f500076
:10500800ecff3e00a02b21009d0807001824a000fb
:10501800100020004f0478000080fa00000006000d
:020000040000fa
:105028000600fa00889fbe008a9fbe0080047800b0
:105038001000200090bf9f000000eb00a0bf9f0061
:10504800b0bf9f00a0bf9f00b91890002fb897006d
:10505800808f50007f0036004a0320000b2020007c
:105068002fb897008a80b9000080440060a890009b
:105078000000e90000004000c160210000804000fd
:10508800100478009880fb00184090004800dd006c
:10509800008070000b006000b0bf9f002fb8970021
:1050a8008a80b9000080440060a8900081af800029
:1050b80092af8000a3af8000b4af8000c5af80007e
:1050c800d6af8000e7af8000c50e07009fb89700f5
:1050d8000100600090bf9f003fb897006000b300d8
:1050e800f0000a00180000002fb897008a80b90065
:1050f8000080440000b0900067406000310020004c
:105108000100dd0071ccb30098c0600000cc7000d5
:10511800284090000040eb0020449800b8409000e0
:10512800304498002fb997008a91b90082804400d2
:10513800b1a89000f13fb2002841900021449800a6
:10514800c808de00b8419000c2cfb30002c16100b8
:1051580081407100314498002fb997008a91b900b5
:1051680082804400a1b0900048499000414c9800ca
:10517800c808de0058499000514c98002fb9970094
:105188008a91b90082804400d1b0900068419000b3
:1051980061449800c808de00784190007144980086
:1051a800c840900040449800d8409000504498006f
:1051b80088489000004c980098489000104c98003f
:1051c8002fb897008a80b900008044006099900049
:1051d8006f4161008848900000cfb30080c0600034
:1051e80082c07000014c98002fb997008a91b900cd
:1051f80082804400e1989000efc060001849900058
:105208000040610001407000104c98002fb89700d2
:105218008a80b90000804400f0a89000efc06000c8
:10522800420020008208dd00084890006f406000be
:1052380001407000004c98002fb897000000e8006b
:10524800a0bf9f00b91890002fb89700808f50001a
:1052580083ff3e001fb897004f05be004f04be00f5
:085268000080fa0000000600be
:020000040000fa
:105270000400fa00889fbe0010002000c0bf9f00fd
:105280008040eb00a1ff9f0064f0b700a0ff9f00eb
:10529000b3c0b300b20621000349780081c0b30057
:1052a000a4062100014a780022c22000328388002f
:1052b00044c0b300d6062100044b78007070ef00a4
:1052c000affc9700e8062100094c7800aff9970081
:1052d000f2062100034978007270ef007170ef0050
:1052e000f5e92400a583880053002000b3838800db
:1052f0007830ef0042062100124178000001610081
:105300004911dd00e67080000690a10006037100df
:10531000e67088004ef0b700a2c0b3005605210029
:10532000024b780048052100014c780006c220009d
:105330008682880076052100044b78005a70ef00c1
:105340005870ef005970ef005c70ef005b70ef0079
:10535000f5828800038388006230ef00e5042100b5
:105360009542780080826200c82add00e6708000e5
:105370000680a10006837200e67088007af0b7000c
:1053800081f0b7008270ef0080f0b700e5c0200028
:10539000e58388008444780038082100094c7800af
:1053a0008670ef008470ef008570ef008870ef006a
:1053b0008770ef00f63f26005684880075002000b5
:1053c000658488000478200074848800a707210081
:1053d0009743780080836300c23bdd00e870800063
:1053e0000820a10008847300e870880090f0b700de
:1053f00029c0b30078092100094c78006709210011
:10540000814b780007c1200097848800990921000a
:10541000824c78009c70ef009a70ef009b70ef0058
:105420009e70ef009d70ef0006858800158588004e
:1054300024858800040921001442780000026200db
:105440000522dd00e57080000570a1008502720074
:10545000e5708800a6f0b70083447800d80a2100e0
:10546000094c780081417800c00a21000348780087
:1054700060c120004085880082427800f40a210043
:10548000054a7800b270ef00b070ef00b170ef0025
:10549000b470ef00b370ef00a6d0bf0000200a0088
:1054a0001c0e00004fb897004f04be000080fa00a9
:0454b00000000600f2
:020000040000fa
:1054b4000600fa00889fbe008a9fbe008c9fbe0033
:1054c4008000eb00f1b79f0012c0b30082f79f0089
:1054d40091bf9f00110020001088a3007e003200bd
:1054e400210020001018a3007b0032001028a30024
:1054f400790032008000eb00f1b79f00b0189000f3
:105504007fb19700828f50006a003600015e21004f
:10551400e48240000182e8008003eb0016c0b3007f
:105524000044eb007fb197004311dd00028140008d
:105534001204e000170032007fb197004311dd0030
:1055440002814000124190000204e0001100320088
:105554007fb197004311dd00028142006055b8001d
:105564000a89be007fb197004311dd0002014200a9
:10557400070978007fb197004311dd0002814000e4
:10558400074978007fb197004311dd000281400094
:1055940017419800ffb19700c319dd000381400053
:1055a40012019000830142008209e800e70f5100d4
:1055b40017003e007fb197004311dd0002814000d7
:1055c400064978007fb197004311dd000281400055
:1055d400184198007fb197004311dd00828140009b
:1055e40023069000b3069000ffb59700fe814500a6
:1055f40083814100830140009301780002814200cd
:105604000c854100e0854e000a89be001800370071
:105614007fb197004311dd00828140002306900092
:10562400b3069000cd6ddd004366de000c86750088
:10563400c36ede00028142000c89be007fb1970078
:105644004311dd0002814000164198007fb19700ac
:10565400ffb19700c319dd00838140002306900049
:10566400b3069000f411b900020140007c219900b6
:105674000ff19700ffb19700c319dd00838140004b
:10568400934190000281fb00030161000201ea00e2
:105694004f11de0082f79f007fb197000201e800fe
:1056a400f2b79f0030199000ffb19700830f5100ab
:1056b4009cff3e000ff097000004e000030032005e
:1056c4001000200090bf9f0002003700200020003f
:1056d40090bf9f009fb89700010078004f06be005e
:1056e4004f05be004f04be000080fa000000060013
:020000040000fa
:1056f4000600fa00889fbe008a9fbe008c9fbe00f1
:1057040010002000f0b79f000000eb0080bf9f0056
:1057140090bf9f008a34ef003816f8009614f90001
:1057240080bf9f000fb897003816e3007100360061
:105734006b9828008a492100e998280064044500f0
:105744008883e90060492100420620006803400084
:105754008001eb000fbe97008fb897008180400056
:1057640081804500ec66b9000c064500110e7800f6
:105774008fbe97008fb897008180400081804400dd
:1057840011067800ec6ab9008400780081004400b6
:105794009c0878000fbe9700ec66b9008c8043002b
:1057a4008fba9700850878008fb897000fbe9700ce
:1057b400ec66b9000c0640002c0690000c06e800cc
:1057c40082e6b9008100e800ec0ab90084007800a0
:1057d400810040008c0878000fbe9700ec66b90089
:1057e4008c0043006022b8008488be0093bf9f00f1
:1057f4000fbe9700ec66b9008c00400031069000a3
:105804009fb89700810f5600330036000fbe9700f3
:10581400ec66b9008c004000110690009fb8970018
:105824008180400081004600110678008fb89700ff
:10583400ec0ab900840078008100400091069000d1
:105844009fb89700818040008180460091007800d5
:10585400910090009fbe9700828ab900840078006e
:105864008d804000211698000fbe9700ec66b900a9
:105874008c004000110690009fb897008180400082
:1058840081004600910078001170a1000fbe9700be
:10589400ec66b9008c004000110690009fb8970098
:1058a4008180400081004600910078001100a10031
:1058b4009fb897008100e80091bf9f000fbe97003a
:1058c400ec66b9008c004000310690009fb8970048
:1058d400810f5600cdff3e008fb897008100e8008d
:1058e40081bf9f008fb89700c5b18000818f52009f
:1058f40098ff3e009c090700ffb09700010060007c
:10590400f0b79f007fb097004f06be004f05be0062
:0c5914004f04be000080fa0000000600f6
:020000040000fa
:105920000400fa00881f78000004780010002000ae
:10593000d0bf9f000000eb000800e0007d003200b7
:10594000486092000004e00018003200401220007d
:10595000080040006e0b07000080fb00e0bf9f00c6
:10596000581091000000e00009003a006fb897005d
:105970000000a20000f0a7000000ea000000e9001b
:105980004f00de00ff000a0018000000070037008b
:105990006fb8970000f0a7000000ea000000e900df
:1059a0004f00de00ff000a00180000001800e000b1
:1059b00006003d001868a30004003a001838a30050
:1059c00002003a001818a3001b003a009800780063
:1059d000618060000004e00005003a001000200033
:1059e00001002000100498002104980004003700f2
:1059f00020002000010020001004980021049800dd
:105a00001800900000004000e15f2100008040008d
:105a1000900078000800780001000100d0bf9f00ce
:105a20005fb8970000f0a7000000ea000000ea005d
:105a30004f00de003f003700180090000a16e30018
:105a400004003e0010002000010020001004980017
:105a5000210498001800900000004000e15f210040
:105a6000808040000000eb001100e00031003200b7
:105a70001800900000004000e15f2100008040001d
:105a8000900078000800780001000100d0bf9f005e
:105a90005fb89700e10f50000b003200030039009f
:105aa000e20f50001b003a001700370010002000e2
:105ab0000100200010049800210498000000eb0071
:105ac000d0bf9f0019003700180090006101b80096
:105ad00012049800230498000000e80010049800c5
:105ae000180090000a16e30004003e002000200089
:105af00001002000100498002104980010002000ec
:105b0000d0bf9f000900370010002000d0bf9f00c9
:105b1000060037001000200001002000100498004b
:105b2000210498008000eb00d1bf9f001810a10055
:105b30005fb897004f0478000080fa00000006006c
:020000040000fa
:105b40000a00fa00889fbe008a9fbe001100200054
:105b5000f1b79f008000eb0081bf9f0091bf9f00c5
:105b6000a1bf9f00b1bf9f0081bf9f00301990006f
:105b70008fb89700810f51006c003600460320005b
:105b8000894c21000800230037ff2f000500280062
:105b9000743821000a0024008b0020000fb9970000
:105ba0008691b90082004000e1989000a1bf9f005b
:105bb000afb897008100e9008180400081804400f7
:105bc00091007800e14190008381fb0071419000d9
:105bd0004811dd000281710002017400e141900072
:105be000e24098004811de00f1419000f240980038
:105bf000814990008381fb00114990004811dd002c
:105c0000028171000701610081499000824898007b
:105c10004811de009149900092489800114190008f
:105c20000274a00092409800414190000234a0000c
:105c3000c24098001181fb00914190004711de00a5
:105c40000e003200031880000381620005003a0054
:105c50001fb997008201e80093bf9f00840f510095
:105c6000f8ff36001fb99700840f510031003e0045
:105c7000031880000301650030003a000fb9970057
:105c80008691b9000201400072c191000204e00057
:105c900003003200c2002000b2bf9f000a0037009c
:105ca0000fb997008691b9000201400042c19100ee
:105cb0000204e0000300320042002000b2bf9f0057
:105cc00001003700bbbf9f00814990008381fb002a
:105cd000114990004811dd0002817100bfb99700a1
:105ce0000301710081499000824898004811de004c
:105cf00091499000924898009140900077810a0065
:105d0000010000007fb1970082806000f1b79f0022
:105d10008fb897008100e80081bf9f003019900084
:105d20008fb89700810f51009cff3e007fb0970015
:105d3000030037000000eb00010037000000eb001b
:105d40004f05be004f04be000080fa0000000600b0
:020000040000fa
:105d50000800fa00881f7800000478001000200076
:105d6000b0bf9f000000eb00c0bf9f00d0bf9f00ee
:105d7000e0bf9f001870a000686890000004e00079
:105d800004003a0010002000b0bf9f003fb8970009
:105d90006c003700a820900008189000808f5000f9
:105da0002800310018209100904090000174a1005b
:105db000114098000000eb00c0bf9f00b818900091
:105dc0004fb89700808f50001b0036004fb89700e7
:105dd000f400b90000004400302891009040900089
:105de0000174a1001140980008007800d400070059
:105df000d0bf9f0018189000dfb8970000804000c7
:105e0000d0bf9f00dfb8970008007800ddf50700dd
:105e1000bfb8970001006000b0bf9f004fb8970067
:105e20000000e800c0bf9f00b81890004fb897006e
:105e3000808f5000e5ff3e0020002000b0bf9f0093
:105e40003f003700a820900008189000808f500075
:105e50003900390028209000401498004810900024
:105e6000d81090000080400040149800281890003e
:105e7000e20f500006003a00381990000820900008
:105e80006102b8000500090042aad800e0bf9f00e7
:105e9000d82191006fb99700182091008000eb0085
:105ea0000300010018209100904090000174a000b0
:105eb0001140980008007800a1000700d0bf9f00a3
:105ec000dfb8970008007800aef50700b0bf9f006c
:105ed00028189000e20f500014003a000000eb0078
:105ee000c0bf9f00b81890004fb89700808f500037
:105ef0000e0036004fb89700f400b90000004400cf
:105f000030289100904090000174a000114098004a
:105f10004fb897000000e800c0bf9f00b81890007d
:105f20004fb89700808f5000f2ff3e001000200015
:105f3000b0bf9f00020037000000eb00b0bf9f0021
:105f40003fb897004f0478000080fa000000060078
:020000040000fa
:105f50000800fa0010002000c0bf9f000000eb0006
:105f6000d0bf9f00e0bf9f00f0bf9f00200cf80053
:105f70004210f9000e0cf8003c10f900100cf8006b
:105f80003e10f900160cf8004610f900e0bf9f0023
:105f9000b18180006fb89700808f50002c003600d0
:105fa000000021008001eb00efb89700fe80400068
:105fb0008180400081004000110178006fba970095
:105fc000f622b90084004000f1809000810f51005a
:105fd00006003100efb89700fe804000818040004d
:105fe00081004000830878000a003700efb897006e
:105ff000fe80400081804000810040001102780056
:106000006fb99700f611b90002014000728190004b
:1060100082085200efb89700fe8040008180400067
:106020008100400011017800ffb897008100410015
:10603000f1bf9f00efb897008100e800e1bf9f002b
:10604000b2818000efb89700810f5100d6ff3e006b
:106050007fb897000000e00002003d000000eb0068
:10606000f0bf9f007fb89700008288005fb897005c
:10607000cfb8970001006000c0bf9f00650c07000b
:10608000cfb8970001006000c0bf9f000000210052
:1060900023fe0700cfb8970001006000c0bf9f003b
:1060a00010808000e30f5000030036002080800045
:1060b000e30f500003003e0010808000e50f500009
:1060c0001a003a00108a8000a06090008180fb00d6
:1060d000306090004800dd0000807000509d880016
:1060e000108a80001040900077800a0000000000b5
:1060f0004f00dd00119d800001f0a10081007000c3
:10610000119d8800108a80001040900077800a005e
:10611000000000004f00dd00519c800001f0a10054
:1061200081007000519c880002003700a3f3a90091
:106130008bf3a9004fb897000080fa00000006001a
:020000040000fa
:106140000200fa0011002000f1bf9f00a01890008b
:10615000e18f50003900320003003900e28f500017
:106160006f003a00380037009020910021519000d4
:106170000281fb00b1509000c808dd008100710071
:106180001800320090209100215990000281fb00fc
:10619000b1589000c808dd00810071001100320084
:1061a00090209100914078000128a30004003a005b
:1061b00090209100914090000148a30009003a000e
:1061c00010209100a05090008180fb003050900082
:1061d0004800dd000080700010007800f0bf9f00d4
:1061e0004d00370090209100a15990008381fb0061
:1061f000315990004811dd00028171008000eb00f0
:106200004800320090209100114190008000eb0086
:106210000248a3004300320010209100a0589000d3
:106220008180fb00305890004800dd000080700045
:1062300010007800f0bf9f003700370070b090006a
:10624000f0bf9f0034003700b0289100215190002a
:106250000281fb00b1509000c808dd008100710090
:1062600018003200b0289100215990000281fb00f3
:10627000b1589000c808dd008100710011003200a3
:10628000b0289100914078000128a30004003a0052
:10629000b0289100914090000148a30009003a0005
:1062a00030289100a05090008180fb003050900079
:1062b0004800dd000080700010007800f0bf9f00f3
:1062c00015003700b0289100a15990008381fb0090
:1062d000315990004811dd00028171008000eb000f
:1062e00010003200b0289100114190008000eb00b6
:1062f0000248a3000b00320030289100a058900003
:106300008180fb00305890004800dd000080700064
:1063100010007800f0bf9f00ffb897000100370021
:106320008000eb00010078000080fa000000060009
:020000040000fa
:106330000200fa0011002000f1bf9f0090009000c1
:1063400081804000421721008100410091007800c7
:10635000300190000200e00010003a00614290001d
:106360000482fb00f1419000c819dd008301720036
:1063700020019000140020000221dd000281ea00cb
:1063800003016100e1419000e24098004811de0005
:10639000f1419000f24098000e00370061429000f9
:1063a0000482fb00f1419000c819dd0083017200f6
:1063b00020019000140020000221dd000281710004
:1063c000e1419000e24098004811de00f141900068
:1063d000f240980040019000e10f51000f003a0098
:1063e000214290000482fb00b1419000c819dd00f9
:1063f0008301720020019000140020000221dd00c2
:1064000002817100a1419000a24098004811de0075
:10641000b1419000b24098000f0037002142900037
:106420000482fb00b1419000c819dd0083017200b5
:1064300020019000140020000221dd000281ea000a
:1064400003016100a1419000a24098004811de00c4
:10645000b1419000b240980040019000e20f51001d
:106460000f003a00014a90000482fb00914990001d
:10647000c819dd0083017200200190001400200083
:106480000221dd000281710081499000824898005c
:106490004811de0091499000924898000f003700a3
:1064a000014a90000482fb0091499000c819dd0068
:1064b0008301720020019000140020000221dd0001
:1064c0000281ea000301610081499000824898003e
:1064d0004811de0091499000924898001182fb001b
:1064e00091419000c819dd008301720020019000e5
:1064f000100020000201dd000281ea0003016100ba
:10650000f0020a0011000000f0bf9f007fb8970062
:086510000080fa000000060003
:020000040000fa
:1065180010f0a6002d0037002014900040159000c0
:106528008608c3008608c1001201c100301b900014
:106538000600c8001a039000260598000a03900078
:10654800160598001001900010d0a7005001900087
:1065580092007800502990000109780010119000ed
:1065680092801000201990008208dd0030149000fd
:10657800010d78008688c3008688c1008688c1001e
:106588001281c100401b90000680c8000000cb00ab
:106598000400cd00402390001620e6000602780093
:1065a8005023900016a0e60006027800100c900018
:1065b800040c7800401590000a0390001605980016
:1065c800040d7800f2320400000000001001900071
:1065d800920078005029900001097800a0389000b6
:1065e800303890000100010000000600801f78008c
:1065f800401090000018eb000008eb004f007800f6
:10660800801f7800501090000018eb000018eb0075
:106618000008eb004f00780000000600801f78009b
:10662800811f780050109000011878000118780038
:1066380001087800cf0078004f007800801f7800ac
:10664800821f780040109000021878000208780035
:106658004f0178004f0078000000060010f0a600f7
:106668001a0037001001900010d0a70050019000c8
:1066780092007800502990000109780010119000cc
:1066880092801000201990008208dd00701b900095
:1066980060199000010278001301c1000200c800cf
:1066a8000400cd00402390001620e6000602780082
:1066b8005023900016a0e60006027800100c900007
:1066c800040c7800723304000000000010019000f0
:1066d8009200780050299000010978000000060017
:020000040000fa
:1066e8000600fa00881f780011002000c1bf9f0033
:1066f8008000eb00d1bf9f00e1bf9f00d1bf9f008a
:1067080030199000dfb89700810f51004f00360014
:1067180043032000874c21000600230035ff2f008b
:1067280004c8b3005fb997008391b90082004000a4
:10673800e1989000e1bf9f00efb897008100e90061
:10674800818040008180430091007800614490007e
:106758000884fb00714190004811dd0002017400bb
:106768000201730061449000e24098004811de0085
:1067780071449000f2409800014c90000884fb009e
:10678800114990004811dd00020174000501610003
:10679800014c9000824898004811de00114c90008e
:1067a800924898001184fb00114190004811dd00c7
:1067b8000201740002f0a100f0020a0011000000ba
:1067c8005fb997008391b9000201400072a190005f
:1067d80041649000c26098004811de005164900046
:1067e800d2609800414490000884fb005141900019
:1067f8004811dd00020174000230a00041449000fd
:10680800c24098004811de0051449000d2409800e0
:106818009140900084c060008180fb008100e90005
:10682800cf08de004fb9970082806000c1bf9f008b
:10683800dfb897008100e800d1bf9f0030199000b1
:10684800dfb89700810f5100b6ff3e00e068920064
:106858000104e00005003200e012b000d403070094
:10686800cfb8970001006000c0bf9f004fb89700e5
:0c6878004f0478000080fa0000000600c9
:020000040000fa
:106884000400fa00889fbe00000478001000200075
:10689400c0bf9f008004eb00d9bf9f0008007800b0
:1068a40020050700cfb8970001006000c0bf9f001b
:1068b4000800780067ed0700cfb89700010060007a
:1068c400c0bf9f001a010700cfb897000100600005
:1068d400c0bf9f00600a20000800400088f607003f
:1068e400cfb8970001006000c0bf9f00e004200003
:1068f4000800400082f60700cfb89700010060004e
:10690400c0bf9f0040062000080040007cf607003e
:10691400cfb8970001006000c0bf9f00d9bf9f009f
:10692400b81890005fb89700808f50000f003600b1
:106934005fb89700f600b900a007b000000044005b
:106944006ff60700cfb8970001006000c0bf9f003a
:106954005fb897000000e800d0bf9f00b81890000f
:106964005fb89700808f5000f1ff3e000800780068
:10697400ac070700cfb8970001006000c0bf9f00bc
:1069840018209100904090000174a10011409800db
:1069940028189000e20f500015003a000000eb00a8
:1069a400d0bf9f00b81890005fb89700808f500048
:1069b400100036005fb89700f400b90000004400ee
:1069c40030289100904090000174a100114098007b
:1069d4005fb897000000e800d0bf9f00b81890008f
:1069e4005fb89700808f5000f2ff3e00010037002f
:1069f4002818900018f0a1001000200001002000c9
:106a040010049800210498004fb897004f04be006a
:086a14000080fa0000000600fa
:020000040000fa
:106a1c001400fa00889fbe00d0bf9f0001047800cc
:106a2c008204780010002000c0b79f000000eb002b
:106a3c00d0b79f00e0b79f006000b800f0b79f0090
:106a4c0081bf9f0090bf9f00a1bf9f00b0bf9f0060
:106a5c00c1bf9f005fb897000000e00003003a0040
:106a6c00800ceb00b91478004a0037001800be0007
:106a7c00f0b79f0081bf9f0021088000d1b79f0015
:106a8c005fb8970000000100cfb0970001006000d4
:106a9c00c0b79f0020088000e0b79f001801be001f
:106aac007fb097008fb8970000005100818059008b
:106abc0090bf9f00a1bf9f001fb89700afb8970071
:106acc00e00f5000e08f580004003200e10f50003e
:106adc00e08f580016003a0007003700efb097001f
:106aec005fb09700008050008000eb00b0bf9f00ab
:106afc00c1bf9f00230037005fb09700f1702200e8
:106b0c00008050008000eb00b0bf9f00c1bf9f0011
:106b1c006fb197003fb89700cfb8970000004100c5
:106b2c00e0804800b0bf9f00c1bf9f001500370038
:106b3c001fb99700afb99700f07022000011b80090
:106b4c00b2bf9f00c3bf9f003fb99700cfb997005a
:106b5c00dfb097000100500000005100e0805900a8
:106b6c00b0bf9f00c1bf9f006fb197003fb89700a7
:106b7c00cfb8970000004100e0804800b0bf9f00f4
:106b8c00c1bf9f003fb89700cfb89700808cbe0064
:106b9c004fb097004f04be000080fa0000000600c2
:020000040000fa
:106bac000a00fa00881f780011002000a1bf9f0086
:106bbc008000eb00b1bf9f0081ff9f00d1bf9f0001
:106bcc00e1bf9f00b1bf9f0030199000bfb8970084
:106bdc00810f51005000360043032000844c2100eb
:106bec000500230007002200060021003fb9970092
:106bfc008391b90082004000e1989000d1bf9f00c2
:106c0c00dfb897008100e9008180400081004200dc
:106c1c00910078003fb997008391b90002014000c0
:106c2c0072c1910082ff9f000ff9970099880a00aa
:106c3c00100000000884ea000281fb0002016400dd
:106c4c000201ea004f11de0082ff9f000ff997004e
:106c5c000204e00002003200e5bf9f00090037008b
:106c6c003fb997008391b9000201400042c19100e5
:106c7c000204e00002003200e6bf9f000100370072
:106c8c00e7bf9f00414190000234a000c240980031
:106c9c00614190000281fb00714490004844dd008a
:106cac00080471006fb997000281ea0008016100c5
:106cbc0061449000e24098004811de00714490005d
:106ccc00f2409800614190000281fb00f14090007d
:106cdc00c808dd00810071006fb997008100610068
:106cec0001f0a7008100ea008100e900cf08de0076
:106cfc002fb9970082806000a1bf9f00bfb897009a
:106d0c008100e800b1bf9f0030199000bfb8970018
:106d1c00810f5100b5ff3e002fb897004f0478004b
:086d2c000080fa0000000600df
:020000040000fa
:106d34000400fa0010002000e0bf9f00bba00a007e
:106d4400a00f0000e0ff9f00a16fa900a40fa900fd
:106d54006ff89700610060004b00dd00017d80004a
:106d640001b0a10081007000017d880001eba90041
:106d740001aba90000062000022bb70002eba9001a
:106d840005eba90005cba900058ba8000070200025
:106d9400042bb70003f82f00205880008080610086
:106da4000100a000215888004100200090210a0021
:106db400060b000007cba90007eba900f1ff210097
:106dc40082b0200012896000098ba900096ba90018
:106dd400094ba900092ba900090ba90008eba9007c
:106de40008cba90001fc2f0080b0200010886000af
:106df40001302800515888000aeba9000a0ba900a9
:106e04000a2ba9000c0ba9000c2ba900c1ff2f0011
:106e1400e2b020001289600031ff2f00e0b02000b2
:106e24001088600000eca900000ca900002ca90047
:106e340000f02000022cb70002eca900020ca9000b
:106e4400022ca9008000eb0090210a00d80b00005e
:106e540090210a00d40b00000230200002007800c8
:106e6400d62bb700b05e8000808061000100a000d6
:106e7400b15e880001c0210001007800d62bb70064
:106e840002007800da2bb700d25e80000280610035
:106e94000000a000d05e880001007800da2bb70063
:0c6ea4006fb897000080fa0000000600a4
:020000040000fa
:106eb0000a00fa00881f780000047800e1bf9f00f4
:106ec00010002000a0bf9f000000eb00b0bf9f009b
:106ed000c0bf9f00a0ff9f006fb89700b0bf9f008a
:106ee0003fb897000000e0002a0032003fb897004a
:106ef0000000e9000000400000004400100078009d
:106f0000c0f50700afb8970001006000a0bf9f0068
:106f10002ff997003fb897000000e90000004000fb
:106f2000000044001000780010007800e1006000cc
:106f30000280fb00010070000000ea004f00de004c
:106f4000a0ff9f003fb897000000e900000040004c
:106f5000000044001000780010007800610160001b
:106f60003fb89700cfb897000281fb000000e9000e
:106f70000010dd0000807000c0bf9f003fb8970088
:106f80000000e900b0bf9f003fb897000000e0009c
:106f9000d6ff3a002ff8970000200a001a160000ca
:106fa0004fb89700e0b088002456e2001700320086
:106fb0002ff897000004e00014003a00f0b08000c1
:106fc00001b180000001e800f2b08800810f50009c
:106fd000080031002216e2000c00320010b18000df
:106fe00000000100afb8970001006000a0bf9f0043
:106ff000060037002016e200040032001a16a8002e
:107000001a36a8002016f8001e16f900aff89700ef
:1070100040622100014878002fb897004f047800a3
:087020000080fa0000000600e8
:020000040000fa
:107028000400fa00881f780000047800100020008f
:10703800d0bf9f000000eb00e0bf9f001870a000c9
:10704800080078008c050700dfb897000100600091
:10705800d0bf9f0028189000e10f500010003200a8
:1070680003003900e20f500042003a0018003700d0
:1070780008007800cbfe0700dfb897000100600029
:10708800d0bf9f0018209100904090000174a0008c
:107098001140980010002000d0bf9f003700370033
:1070a80008007800bffe0700dfb897000100600005
:1070b800d0bf9f0018209100904090000174a0005c
:1070c8001140980010002000d0bf9f002b0037000f
:1070d800686890000004e0001e003a00080078008c
:1070e800b0fe0700dfb8970001006000d0bf9f0026
:1070f80018209100904090000174a0001140980061
:107108000000eb00e0bf9f00b81890006fb8970030
:10711800808f5000140036006fb89700f400b90053
:107128000000440030289100904090000174a000b5
:10713800114098006fb897000000e800e0bf9f007a
:10714800b81890006fb89700808f5000f2ff3e008b
:10715800050037000800780092fe0700dfb89700a6
:1071680001006000d0bf9f0010002000d0bf9f002a
:10717800020037000000eb00d0bf9f005fb8970007
:0c7188004f0478000080fa0000000600b0
:020000040000fa
:1071940010f0a6003800370020149000401590002d
:1071a4008608c3008608c1001201c100301b90008c
:1071b4000600c8001a039000260598000a039000f0
:1071c400160598001001900092007800400190008c
:1071d400810011001011900092801000201990007d
:1071e4008208dd0030149000010d78008688c30009
:1071f4008688c1008688c1001281c100401b9000ae
:107204000680c8000000cb000400cd00402390009d
:107214001620e600060278005023900016a0e6002f
:1072240006027800100c9000040c78008011900085
:1072340083014200500c9000030c780041a3de004f
:10724400302c900008054300202c90000a0c780094
:10725400102c900008054300002c90000a0c7800c4
:10726400401590000a03900016059800040d78005c
:1072740042390400000000001001900092007800e0
:1072840000000600801f7800401090000018eb00fa
:107294000008eb004f007800801f78005010900029
:1072a4000018eb000018eb000008eb004f0078001a
:1072b40000000600801f7800811f780050109000a5
:1072c400011878000118780001087800cf007800d0
:1072d4004f007800801f7800821f780040109000d3
:1072e40002187800020878004f0178004f007800f7
:0472f4000000060090
:020000040000fa
:1072f8001400fa00f0bf9f0010002000e0b79f00c4
:10730800f0b79f00a0bf9f007fb89700c10320007f
:10731800810f5000290032000d003e00fe0f500082
:107328001d00320003003e00f40f500043003a00f5
:107338001600370081022000810f5000190032002a
:10734800ea804000810f50003c003a0018003700e6
:1073580001052000810f50001e00320004003e008d
:10736800ea805000810f500034003a0016003700c0
:10737800a1052000810f500019003200ea8040006a
:10738800810f50002d003a001800370040012000fe
:10739800b0bf9f0017003700e0012000b0bf9f007a
:1073a8001400370080022000b0bf9f001100370092
:1073b80020032000b0bf9f000e003700c00320004c
:1073c800b0bf9f000b00370060042000b0bf9f00d3
:1073d8000800370000052000b0bf9f0005003700f7
:1073e800a0052000b0bf9f00020037004006200023
:1073f800b0bf9f0020002000c0bf9f0010002000e9
:10740800d0bf9f007fb097008fb897001fb9970033
:10741800afb997003fba9700cfba97005fbb970004
:10742800efbb970021f50700efb09700010060005f
:10743800e0b79f006fb09700010037000000eb0035
:087448000080fa0000000600bc
:020000040000fa
:107450000600fa0011002000d1bf9f008000eb0061
:10746000e1bf9f00e1bf9f0030199000efb8970087
:10747000810f51003a00360046032000854c210060
:10748000040023008041eb006fb997008691b9009a
:1074900082004000e1989000f1bf9f00ffb8970084
:1074a0008100e900818040008180420091007800e5
:1074b000e14390008783fb00714190004811dd009b
:1074c0000281730002017200e1439000e2409800e3
:1074d0004811de00f1439000f240980041619000b5
:1074e000c360980051619000d3609800c143900040
:1074f0008783fb00514190004811dd000281730039
:107500000230a000c1439000c24098004811de0044
:10751000d1439000d2409800614190000281fb006d
:10752000f1409000c808dd00810071008480600097
:107530008100ea00cf08de005fb99700828060001a
:10754000d1bf9f00efb897008100e800e1bf9f0026
:1075500030199000efb89700810f5100caff3e002c
:10756000e06892000104e00005003200e012b00083
:1075700091000700dfb8970001006000d0bf9f00b6
:0c7580005fb897000080fa0000000600d1
:020000040000fa
:10758c000400fa00881f7800000478001000200026
:10759c00d0bf9f000000eb00e0bf9f0018209100bf
:1075ac00904090000174a10011409800b820910007
:1075bc00182091000100010028189000e20f5000e3
:1075cc001d003a000000eb00e0bf9f00b8189000cf
:1075dc006fb89700808f5000170036006fb8970077
:1075ec00f400b90000004400302891009040900055
:1075fc000174a100114098006fb89700f400b90015
:10760c0000004400d02891006fb89700f400b90036
:10761c000000440030289100010001006fb8970071
:10762c000000e800e0bf9f00b81890006fb897000a
:10763c00808f5000e9ff3e00080078003df90700fc
:10764c00dfb8970001006000d0bf9f005fb89700c3
:10765c000000e000010032001820a0002818900063
:10766c00e10f500005003a000800780044030700c1
:10767c00dfb8970001006000d0bf9f0095020700a3
:10768c00dfb8970001006000d0bf9f0018f0a00089
:10769c001000200001002000100498002104980024
:1076ac005fb897004f0478000080fa0000000600d5
:020000040000fa
:1076bc000400fa0012002000e2bf9f008000eb00e3
:1076cc00f1bf9f0090009000818040004317210083
:1076dc008180410091007800a00190000311dd0031
:1076ec00f2bf9f00300090000000e0000d003a0057
:1076fc00614190000281fb00714090004800dd0068
:10770c00000071007fb99700020070006141900089
:10771c00e04098004800de0071419000f040980075
:10772c000d003700e14190008381fb007141900016
:10773c004811dd00028171007fb897000080ea00db
:10774c000200600061419000e04098004800de00bb
:10775c0071419000f0409800e14190008381fb0062
:10776c00714190004811dd0002817100c14190000f
:10777c008381fb00514090004800dd0000807100c7
:10778c00ffb89700020068000100600000f0a7003d
:10779c000000ea000000e9004f00de00e0bf9f009f
:0c77ac006fb897000080fa000000060093
:020000040000fa
:1077b8000400fa0012002000e2bf9f008000eb00e6
:1077c800f1bf9f0090009000818040004317210086
:1077d8008180410091007800a00190000311dd0034
:1077e800f2bf9f00300090000000e0000e003a0059
:1077f800e14190008381fb00714190004811dd0058
:10780800028171007fb897000080ea0002006000e2
:1078180061419000e04098004800de00714190000e
:10782800f04098000c003700614190000281fb0095
:10783800714090004800dd00000071007fb997009a
:107848000200700061419000e04098004800de00ae
:1078580071419000f0409800e14190008381fb0065
:10786800714190004811dd0002817100c141900012
:107878008381fb00514090004800dd0000807100ca
:10788800ffb89700020068000100600000f0a70040
:107898000000ea000000e9004f00de00e0bf9f00a2
:0c78a8006fb897000080fa000000060096
:020000040000fa
:1078b4000200fa00881f7800000478000000eb0042
:1078c400e0bf9f0028009000de15e30002003e00a8
:1078d4000000eb0020049800280090000000400005
:1078e400015d2100808040000000eb001100e000f9
:1078f4002a0032002800900000004000015d2100b1
:107904000080400090007800080078000100010029
:10791400e0bf9f006fb89700e10f500004003200f1
:10792400e20f50001a003a00e0bf9f001a0037002f
:10793400280090000000e80020049800280090002f
:10794400de15e3000f00360020002000e0bf9f009a
:1079540028009000e50f50000f003a00281890000e
:107964000000e0000300320028189000e10f5000ee
:1079740009003a00280090000000e8002004980064
:107984000500370010002000e0bf9f000200370010
:107994000000eb00e0bf9f006fb897004f04780031
:0879a4000080fa00000006005b
:020000040000fa
:1079ac000200fa008000eb00f1bf9f001070a000f5
:1079bc00a0189000e28f500028003a00902091000f
:1079cc00a1c990008381fb0031c990004811dd00f2
:1079dc00028171008011900003014100a1c9900047
:1079ec00a2c898004811de00b1c99000b2c8980036
:1079fc00d00890008100e800510898009020910078
:107a0c00a1c990008381fb0031c990004811dd00b1
:107a1c0002817100d0189000810f51000c003900c8
:107a2c00d018900001209900902091000020910026
:107a3c0021c99000a0c898004800de0031c9900010
:107a4c00b0c8980010002000f0bf9f000c00370059
:107a5c0020002000f0bf9f0009003700902091000b
:107a6c000020910021c99000a0c898004800de00b9
:107a7c0031c99000b0c8980010002000f0bf9f00e2
:0c7a8c007fb897000080fa0000000600a0
:020000040000fa
:107a98000c00fa00a0bf9f00b1bf9f00c2bf9f00ab
:107aa800d3bf9f00e4bf9f00f5bf9f006fb897004a
:107ab800630060004800dd00f1cf2f00927c800059
:107ac8008280600081007000917c8800f0032000b3
:107ad800afb897000080600050200a008e0f0000a9
:107ae8003fb89700b0200a00900f00004fb89700e9
:107af800670060004400dd00f1f82f00927c8000f0
:107b08008280600081007000917c88005fb89700d7
:107b180020200a00920f00007fb8970061006000e3
:107b28004800dd00717c80000180a10081007000a8
:107b3800717c88007fb8970022800a00000000004e
:107b48004f00dd00717c800001f0a1008100700011
:107b5800717c8800ffb897000000eb000128a300a3
:107b680004003200707c8000ff800a0000000000e2
:0c7b78000080fb000080fa000000060006
:020000040000fa
:107b84000200fa0010002000f0bf9f00e08588008a
:107b9400f0858800e100200001868800f1002000c3
:107ba40011868800c570ef00c6f0b700c7f0b700b3
:107bb400c470ef0005f4210045868800ca30ef0048
:107bc400820c20007286880062868800045e210090
:107bd40084868800f980400091868800a186880008
:107be400031e2000b3868800da30ef00c0868800c8
:107bf4004600200086878800908788006600200061
:107c0400a687880056002000b6878800f970ef0028
:107c1400faf0b700fbf0b700f870ef00e5878800d2
:107c240005fa2000f58788001288880002888800f9
:107c34002488880031888800418888005388880017
:107c44000e31ef00608888007fb897000080fa004a
:047c54000000060026
:020000040000fa
:107c58000200fa00881f7800000478000000eb009a
:107c6800e0bf9f001800e00003003d0018e8a300f3
:107c78000100320018d0a0008000eb000800780056
:107c8800a1030700e0bf9f006fb89700e10f500005
:107c980003003200e20f50000b003a0006003700e4
:107ca8001850a0001870a100200020001800e00063
:107cb80009003500170037001850a1001870a000ff
:107cc80020002000130037001850a1001870a100f0
:107cd8000000eb000f0037002000200018d8a30098
:107ce8000c0032001818a3000a0032001828a3005c
:107cf800080032001838a30006003a001868a300ec
:107d080004003a001858a3000200320018d0a1005d
:107d1800100020004f0478000080fa0000000600e0
:020000040000fa
:107d28000400fa00889fbe0080047800100020003c
:107d3800000f7800bba00a00a00f000020479800a1
:107d4800a16fa900a52fa9002e4090006100600036
:107d58004b00dd00017d800001b0a10081007000b2
:107d6800017d88002be3a90061e3a90097e3a9003e
:107d7800cde3a90003e4a90039e4a9006fe4a90050
:107d8800a5e4a900af02b00068fd2f000f0444006d
:107d9800a042210029000900305c7800a802b10047
:107da800e90407001e0f600059c091008807780099
:107db8000004e00007003200c9a090000030200055
:107dc8002049900021489800c808de0030499000fa
:107dd800314898001e0078004f04be000080fa0069
:047de8000000060091
:020000040000fa
:107dec000400fa00881f78000004780010002000be
:107dfc00d0bf9f000000eb00e0bf9f0008007800a0
:107e0c0036fa0700dfb8970001006000d0bf9f0072
:107e1c0018209100904090000174a100114098002e
:107e2c0028189000e20f500014003a000000eb00fc
:107e3c00e0bf9f00b81890006fb89700808f50007b
:107e4c000e0036006fb89700f400b9000000440033
:107e5c0030289100904090000174a10011409800ce
:107e6c006fb897000000e800e0bf9f00b8189000c2
:107e7c006fb89700808f5000f2ff3e0018f0a10001
:107e8c00100020000100200010049800210498002c
:107e9c005fb897004f0478000080fa0000000600dd
:020000040000fa
:107eac000200fa008000eb00f1bf9f003100980047
:107ebc00010898001010a100a01890000100e0002b
:107ecc0002003a001050a000050037001088a300f3
:107edc00020032001050a100010037001050a00029
:107eec0090209100114190000274a10092409800e2
:107efc00a0189000e28f500014003a008000eb00b4
:107f0c00f1bf9f00b01890007fb99700828f50008e
:107f1c000e0036007fb99700f411b90082004000c2
:107f2c00b1289100114190000274a1009240980078
:107f3c00ffb897008100e800f1bf9f00b0189000d7
:107f4c007fb99700828f5000f2ff3e001070a100a5
:107f5c001000a000100020000080fa0000000600b5
:020000040000fa
:107f6c000200fa0010002000f0bf9f00001020005b
:107f7c00904090000174a100114098009040900036
:107f8c000154a10011409800904090000144a100c0
:107f9c0011409800904090000134a10011409800cd
:107fac00904090000124a100114098009040900056
:107fbc003140b300114098001074a100f1ccb30013
:107fcc0010c860001024a1001014a100c040900043
:107fdc008040eb0041409800504190005140980087
:107fec0080489000f1c0b300014898009048900080
:107ffc0071c2b30011489800f0f82f004008b60089
:10800c000050a000004288000028a9002028a900e8
:0c801c007fb897000080fa00000006000a
:020000040000fa
:108028000400fa0010002000e0bf9f000000eb00f1
:10803800f0bf9f000010a9000030a9000050a9005f
:108048000070a8000090a9000110a9000130a90043
:1080580001d0a80001f0a90000d0a800110020005c
:10806800118088000430ef0021002000a1818800e1
:10807800423d2000d28188000281e900c281880047
:10808800b1818800f0bf9f00b18180007fb8970060
:10809800808f5000090036000001eb00e281880063
:1080a8007fb897000000e800f0bf9f00b181800012
:1080b8007fb89700808f5000f8ff3e004030ef00f7
:1080c8004430ef004230ef004630ef006fb89700c1
:0880d8000080fa000000060020
:020000040000fa
:1080e0000600fa0010002000d0bf9f000000eb0047
:1080f000e0bf9f00f0bf9f0001eba800f10f200040
:1081000070b18000010060000060880070b18000e4
:108110004800dd002e16b700f0bf9f0015c0b30069
:1081200074a923000043eb0002608000ffb89700b1
:108130006fb897008001e800e3bf9f00810f5100f6
:108140000600320085407800840f500001003600a0
:10815000864078000104e000f3ff3a006fb9970011
:108160000000eb0071a92300810f510006003e00c2
:1081700000f02f000a2bb60070b180000080fb00d9
:108180000a2bb7005fb897000080fa0000000600d5
:020000040000fa
:108190000200fa00881f780010002000e0bf9f0056
:1081a00008c8200061622100914078008180fb00b6
:1081b00027d6bf004800dd000080700082622100e9
:1081c000124178000281fb00916221009140780009
:1081d000c808dd0081007100a3622100934178008e
:1081e0008381fb00b2622100124178004811dd005a
:1081f00002817100c4622100144278000482fb00f5
:10820000d362210093417800c819dd008301720018
:108210004c030700efb8970001006000e0bf9f002b
:10822000184090000074a100104498006fb89700a7
:0c8230004f0478000080fa0000000600f7
:020000040000fa
:10823c000400fa00889fbe0010002000c0bf9f0001
:10824c000000eb00d0bf9f0027f50700cfb89700c8
:10825c0001006000c0bf9f00b0010700cfb89700bd
:10826c0001006000c0bf9f008a14e20016003500b8
:10827c0009002800f85227003656e20005003200ab
:10828c005fb897008000e800d1bf9f00880f5000b6
:10829c00f9ff3600110020002000200016ef070027
:1082ac00cfb8970001006000c0bf9f000000eb003a
:1082bc00d0bf9f0010c0b30036f6b70051a48000a9
:1082cc0001806400ecff32000000fe000000eb00b7
:0c82dc004f04be000080fa000000060005
:020000040000fa
:1082e8000200fa0010002000f0bf9f0000002100eb
:1082f80062f90700ffb8970001006000f0bf9f0017
:1083080022cea9001ecea90022aea9001eaea90049
:10831800a2030700ffb8970001006000f0bf9f00ac
:1083280021c2b30060c2b30013020700ffb8970070
:1083380001006000f0bf9f0031c2b30050c2b3001b
:108348000d020700ffb8970001006000f0bf9f0012
:108358009c030700ffb8970001006000f0bf9f0072
:10836800901a80004200de00a01a8800901a80004f
:108378004200de00a01a88007fb897000080fa004b
:0483880000000600eb
:020000040000fa
:10838c000400fa008000eb00e1bf9f001200200007
:10839c00f2bf9f00e1bf9f00b01890006fb997002b
:1083ac00828f50001700360044032000c360210068
:1083bc006fb997008491b90082004000e1a8900049
:1083cc008100e900818040008180410091007800ab
:1083dc00314990000274a000b248980011419000fd
:1083ec000274a00092409800efb897008100e8005a
:1083fc00e1bf9f00b01890006fb99700828f5000ba
:10840c00ebff3e0000c82000904090000174a000db
:10841c00114098007fb897000080fa000000060019
:020000040000fa
:10842c000200fa0010002000f0bf9f00fbfe0700c6
:10843c00ffb8970001006000f0bf9f00cefd070061
:10844c00ffb8970001006000f0bf9f0078020700a2
:10845c00ffb8970001006000f0bf9f0081f3070098
:10846c00ffb8970001006000f0bf9f005d0007009f
:10847c00ffb8970001006000f0bf9f00a8e3070061
:10848c00ffb8970001006000f0bf9f0093ff07004a
:10849c00ffb8970001006000f0bf9f00500207007a
:1084ac00ffb8970001006000f0bf9f007fb89700f5
:0884bc000080fa000000060038
:020000040000fa
:1084c40040199000c0189100810f51001f00320024
:1084d4001070a00040199000c0189100810f510045
:1084e4000b00310040199100d01090008100510020
:1084f4004118990040199100c0189000810f510053
:1085040013003100c0189000411899001000370082
:1085140040199000c0189100810f51000c003600e2
:10852400c018910050119000810041004118990039
:1085340040199100c0189000810f510004003600ca
:10854400c018900041189900010037001070a10074
:088554002000200000000600d9
:020000040000fa
:10855c001000fa00f0bf9f001000200080bf9f00a9
:10856c006fb897000000a000e0bf9f000000eb0078
:10857c00d0bf9f007fb9970001322000810f5100be
:10858c0016003e001000200090bf9f00ffb897001f
:10859c00c208de00a1bf9f0021002000b1bf9f00d8
:1085ac00c0bf9f006fb897000020a000e0bf9f00e5
:1085bc001fb89700afb897003fb99700cfb9970095
:1085cc005fba9700efba970030fd07008fb897009d
:1085dc000100600080bf9f000fb897000080fa0078
:0485ec000000060085
:020000040000fa
:1085f0000200fa0010002000f0bf9f00f07c200075
:1086000040808800703e2000308188002a30ef00d2
:108610002830ef002c30ef00a0818000e20f5000e6
:108620000d003a002830ef00d00d20006081880056
:10863000713e2000e18088002030ef001e30ef0006
:108640002230ef0013c0b300e2022100034978009a
:1086500080818800030037002e70ef00203d20004d
:1086600080818800f07c200090808800203d2000e0
:10867000a08088007fb897000080fa000000060004
:020000040000fa
:108680000600fa0011002000d1bf9f008000eb001f
:10869000e1bf9f00f1bf9f00e1bf9f003019900034
:1086a000efb89700810f51001600360044032000f8
:1086b000834c21006fb997008491b900820040007b
:1086c000e1989000f1bf9f00ffb897008100e9009a
:1086d00081804000818041009100780041419000fc
:1086e0000234a000c2409800efb897008100e80073
:1086f000e1bf9f0030199000efb89700810f510043
:10870000ecff3e005fb897000080fa000000060012
:020000040000fa
:108710000200fa0011c0b300e1ff9f00900090003a
:1087200081804000421721008100410091007800c3
:10873000c14190008381fb00514190004811dd0050
:1087400002817100a0009000130020008118dd005c
:108750008280600001f0a7008100ea008100ea0049
:10876000cf08de00e1ff9f0030009000830f500033
:1087700008003a00eff897000180fb0000805100ec
:1087800000f0a7000000ea000000ea004f00de0051
:10879000e0ff9f006ff897000080fa0000000600dd
:020000040000fa
:1087a0000400fa00e0ff9f00f1ff9f00100020008e
:1087b000e0bf9f007ff89700670060004400dd0085
:1087c000f1f82f000242800082806000810070007a
:1087d000014288000028a9006ff89700610060003e
:1087e00000004000014180000110a10081007000e4
:1087f0000141880000102000904090000174a0000a
:10880000114098001040900077800a00000000009e
:10881000efb8970001006000e0bf9f006fb89700bd
:088820000080fa0000000600d0
:020000040000fa
:108828000200fa00881f7800000478001000200079
:10883800e0bf9f00486092000004e000040032009e
:108848004012200008004000b7f60700e0bf9f0074
:10885800686892000004e00004003200e012200082
:1088680008004000b0f60700e0bf9f00686892006b
:108878000004e00006003200e0122000080040007a
:10888800cbfb0700efb8970001006000e0bf9f0036
:108898006fb897004f0478000080fa0000000600c7
:020000040000fa
:1088a8000200fa0011002000f1bf9f001070a00024
:1088b800c0109000501190008100410041109800b4
:1088c800a01090008100e80021109800401190004d
:1088d800c0189100810f51000c003600c01891009b
:1088e80041109800902091008013b0002161900001
:1088f800a06098004800de0031619000b0609800e8
:1089080010002000f0bf9f00020037002000200068
:10891800f0bf9f007fb897000080fa0000000600b3
:020000040000fa
:108928000200fa00881f780018002000e8bf9f00a6
:108938008040eb000140780097ff0700efb89700f0
:1089480001006000e0bf9f008000eb00010078009c
:108958006aed0700efb8970001006000e0bf9f00d4
:108968008000eb000800780064ed0700efb897007e
:1089780001006000e0bf9f0021c0b30008407800fc
:1089880085ff0700efb8970001006000e0bf9f0077
:108998006fb897004f0478000080fa0000000600c6
:020000040000fa
:1089a8000200fa008000eb00f1bf9f001070a000e9
:1089b80080089000100990008101e80003089800e1
:1089c800828f500010003600900890008100e80067
:1089d80001089800e06892000104e00007003200f6
:1089e800e012b00033fb0700f0bf9f000000eb006f
:1089f800ffb897000100e0000600320010002000d8
:108a0800f0bf9f000200370020002000f0bf9f0049
:0c8a18007fb897000080fa000000060004
:020000040000fa
:108a24000200fa00881f780000047800100020007b
:108a3400e0bf9f000800780084fa0700efb89700b1
:108a440001006000e0bf9f000800780009ec070007
:108a5400efb8970001006000e0bf9f000000eb004a
:108a640030049800000c9800500c980020149800d2
:108a74001810a1001870a1006fb8970000f0a700ab
:108a84000000ea000000ea004f00de004f04780016
:088a94000080fa00000006005a
:020000040000fa
:108a9c000600fa00f1bf9f0011002000d1bf9f001b
:108aac008000eb00e1bf9f00e1bf9f006fb9970012
:108abc00ffb89700810f51000f003100efb89700fd
:108acc00818040008100400091007800a257210075
:108adc000b000900b21878008101b100efb89700c3
:108aec008100e800e1bf9f006fb99700ffb89700c5
:108afc00810f5100f1ff39005fb897000080fa0038
:048b0c00000006005f
:020000040000fa
:108b10000400fa00f1bf9f008000eb00e1bf9f005e
:108b20000000e000130032007fb99700a3b180007d
:108b3000828f51000f003600ffb8970081804000ff
:108b400022632100010141008000eb001200e000df
:108b500008003200ffb897008180400022632100a6
:108b6000810041009100780001000100e0bf9f00fa
:108b7000efb89700010078000080fa0000000600be
:020000040000fa
:108b80000600fa00e0ff9f00f1ff9f000000eb00ed
:108b9000d0bf9f00c0ff9f00eff8970000ceb3004a
:108ba00000c04000c0ff9f004ff897000080fb000e
:108bb00001d8200000804000fff8970001487800ad
:108bc000904078007ff8970000c068000080fb00ac
:108bd0000000e9004f00de00d0bf9f005fb89700a3
:088be0000080fa00000006000d
:020000040000fa
:108be8001200fa0080bf9f0091bf9f00a2bf9f00a4
:108bf800b3bf9f00c4bf9f00d5bf9f00e6bf9f00c3
:108c0800f7bf9f0010002000f0b79f000fb8970033
:108c18000000e90000004000c16021000080400021
:108c280010007800ee8057000d00090031587800d8
:108c3800e000b1007fb097000080fa000000060055
:020000040000fa
:108c48000200fa0010002000f0bf9f00e4000700b7
:108c5800ffb8970001006000f0bf9f00a800070060
:108c6800ffb8970001006000f0bf9f005e01070099
:108c7800ffb8970001006000f0bf9f009100070057
:108c8800ffb8970001006000f0bf9f007fb8970011
:088c98000080fa000000060054
:020000040000fa
:108ca0000200fa00881f7800000478000000eb0042
:108cb000e0bf9f0008007800e5f90700e0bf9f00d3
:108cc0001870a1006fb897000000e00003003200a8
:108cd00010002000e0bf9f00020037000000eb0002
:108ce000e0bf9f006fb897004f0478000080fa0043
:048cf000000006007a
:020000040000fa
:108cf4000200fa008000eb00f1bf9f001070a0009a
:108d0400b0009000400190008101e8003300980019
:108d1400828f500006003600c00090008100e800f9
:108d24003100980010002000f0bf9f0002003700bf
:108d340020002000f0bf9f007fb897000080fa0059
:048d44000000060025
:020000040000fa
:108d48000400fa00f0bf9f0010002000e0bf9f0061
:108d58007fb897000000e90000004000814c210026
:108d680000804000900078000000eb000100e00067
:108d78000600320000fc2f00008047003500090083
:108d8800b05878006103b1006fb897000080fa000e
:048d980000000600d1
:020000040000fa
:108d9c000200fa0010002000f0bf9f00219e80000e
:108dac00a03b21003ff80700d0b0800061006000bc
:108dbc004300dd00018080000130a10081007000c3
:108dcc000180880010808000e50f500001003a00ff
:108ddc001e36ef007fb897000080fa0000000600f6
:020000040000fa
:108dec000200fa0010002000f0bf9f00202ba8000a
:108dfc00f02ba80080ff2f006e08b6005000b300c7
:108e0c00704388000b88a9002b88a800cca00a000e
:108e1c002a0800000080fb00ffb8970001006000ea
:108e2c00f0bf9f007fb897000080fa00000006009a
:020000040000fa
:108e3c000200fa0011002000f1bf9f002471ef0026
:108e4c0020002000308988005200200042898800d0
:108e5c002a31ef00618988002e71ef00808988002b
:108e6c0040002000908988003431ef003631ef004b
:0c8e7c007fb897000080fa00000006009c
:020000040000fa
:108e88004213a8004233a80043f3a8005a13a800cd
:108e98005a33a8005bf3a8007213a8007233a80025
:108ea80073f3a8008a13a9008a33a9008bf3a900d9
:108eb800a213a900a233a900a3f3a900100020005f
:048ec80000000600a0
:020000040000fa
:108ecc00400420001040a1001000a1001010a100cf
:108edc001070a0001060a0001050a100f1ff2c0039
:108eec001088600010f0a1000000000000000000dd
:0c8efc0000000000100020000000060034
:020000040000fa
:108f08000200fa0010002000f0bf9f00401f200060
:108f180090fd0700ffb8970001006000f0bf9f00b8
:108f2800abe50700ffb8970001006000f0bf9f00a5
:0c8f38007fb897000080fa0000000600df
:020000040000fa
:108f44000a00fa00c0bf9f00d1bf9f00e2bf9f008c
:108f5400f3bf9f0010002000b0bf9f0000c8200096
:108f6400e880570007000900315878003fb897009f
:088f74000080fa000000060075
:020000040000fa
:108f7c000200fa0010002000f0bf9f002fff070036
:108f8c00ffb8970001006000f0bf9f00a8fc07002d
:108f9c00ffb8970001006000f0bf9f000000eb00dd
:088fac000080fa00000006003d
:020000040000fa
:108fb400b0ac88009835ec00000000000000000010
:108fc400000000000000000000000000000000009d
:108fd4009215ab00020032009435ec000000fe0054
:048fe4000000060083
:020000040000fa
:108fe8000200fa0010002000f0bf9f004006200099
:108ff800bff80700f0bf9f0075e50700ffb89700ae
:1090080001006000f0bf9f007fb897000080fa0061
:04901800000006004e
:020000040000fa
:10901c000200fa0010002000f0bf9f0060862400c0
:10902c0010b188004000200000b188001e36ef000f
:0c903c007fb897000080fa0000000600da
:020000040000fa
:109048000200fa0010002000f0bf9f00000021007d
:109058004cf90700ffb8970001006000f0bf9f00bf
:0c9068007fb897000080fa0000000600ae
:020000040000fa
:109074000200fa0010002000f0bf9f000000210051
:1090840059fb0700ffb8970001006000f0bf9f0084
:0c9094007fb897000080fa000000060082
:020000040000fa
:1090a0000200fa0010002000f0bf9f000000210025
:1090b00011000700ffb8970001006000f0bf9f009b
:0c90c0007fb897000080fa000000060056
:020000040000fa
:1090cc000200fa000000eb00f0bf9f00000021003e
:1090dc0011000700ffb8970001006000f0bf9f006f
:0c90ec007fb897000080fa00000006002a
:020000040000fa
:1090f8000200fa0011002000f1bf9f001060a000dc
:1091080005f20700ffb8970001006000f0bf9f005c
:0c9118007fb897000080fa0000000600fd
:020000040000fa
:109124000200fa0011002000f1bf9f001060a100ae
:10913400faf10700ffb8970001006000f0bf9f003c
:0c9144007fb897000080fa0000000600d1
:020000040000fa
:109150000200fa0010002000f0bf9f000030200045
:10916000e1fc2f0081804700290009003158780078
:0c9170007fb897000080fa0000000600a5
:020000040000fa
:10917c000200fa0010002000f0bf9f00a8fc0700be
:10918c00ffb8970001006000f0bf9f007fb8970008
:08919c000080fa00000006004b
:020000040000fa
:1091a4000000eb0051052000b1468800a10a200010
:1091b400b146880000688800bba00a00000d0000ca
:0891c40061001000000006002c
:020000040000fa
:1091cc000080200051052000b1468800a10a200033
:1091dc00b146880000688800bba00a00000d0000a2
:0491ec000000060079
:020000040000fa
:1091f0000200fa0010002000f0bf9f00002eef00d8
:109200001c2eef00382eef007fb897000080fa0088
:049210000000060054
:020000040000fa
:109214000400fa0010002000e0bf9f008000eb0073
:0c922400f1bf9f000080fa00000006006f
:020000040000fa
:10923000219e8000a03b210018fe070010002000a6
:049240000000060024
:020000040000fa
:020000040005f5
:047e0000ffffff0081
:020000040000fa
:020000040005f5
:047e2000ffffff0061
:020000040000fa
:020000040005f5
:047e30007fffff00d1
:020000040000fa
:020000040005f5
:047e38007be7ff00e5
:020000040000fa
:020000040005f5
:047e4000677fff0059
:020000040000fa
:020000040005f5
:047e4800ffffff0039
:020000040000fa
:020000040005f5
:047e5000deffff0052
:020000040000fa
:020000040005f5
:047e58000000ff0027
:020000040000fa
:020000040005f5
:047e60000000ff001f
:020000040000fa
:020000040005f5
:047e68000000ff0017
:020000040000fa
:020000040005f5
:047e70000000ff000f
:020000040000fa
:020000040005f5
:047e7800ffffff0009
:020000040000fa
:020000040005f5
:047e8000fffcff0004
:020000040000fa
:020000040005f5
:047e8800c9ffff002f
:00000001FF
